:020000041100E9
:103000007FB50023284C294D03932800217C284AB2
:1030100001F0D3FA002812D103232800217C03AA4F
:1030200001F072FA00280AD1224B039A9A4206D183
:10303000214B2248E360224B636104B070BD02263D
:10304000217CFE2228001F4B009601F02FFA002859
:1030500001D00020F1E71C4BA2899A42F9D1217CD2
:10306000FF222800194B009601F020FA0028F0D129
:10307000E389174A934203D1164B17486361DCE793
:10308000164A9342E5D1164B164A1B68934206D95D
:10309000C02304222800217C9B0001F070FA124B0F
:1030A00012486361C9E7C046AC61FF1FDC41FF1FE6
:1030B000813700005959530059598320CCBE001163
:1030C000ED410011B861FF1F59590000BA61FF1F9F
:1030D00083050000A1410011ACBE00118215000063
:1030E000D061FF1F87130000A9420011BCBE001170
:1030F000002370B51A4E1B4C30006361637401F0FD
:1031000083F9402323744B2B0CD9CC233821AC22D8
:1031100030009B01217401F032FA00280AD000250A
:1031200025740CE0FFF76CFF051E08D1237C0433E7
:10313000DBB2E7E70C4B0D4D63610D4BE381236878
:10314000002B08D1002D06D00C222900200008F009
:10315000E7FD2B7B6374300001F094F970BDC0462D
:10316000DC41FF1FAC61FF1F414200119CBE0011FA
:10317000AAAAFFFFF7B5164B0192C318021D002043
:10318000009388235B05D3181B685C1C1AD09CB283
:10319000402C18D88D781E0CAC466746CD782D0291
:1031A0003D43AE4206D1019800280ED110000C70AC
:1031B000240A4C7003249BB20733A343D218009B0C
:1031C0009A42DED3FEBD4432F9E71000FAE7C0466A
:1031D000FC0F0000802213B503000324019189B283
:1031E000520107319B18A14304305A1A88235B050A
:1031F000C3181B68591C03D190429241104016BD60
:1032000099B2402907D80B000733A343C018904256
:10321000ECD30020F3E74430F9E7134B134A1B6863
:10322000126810B5FA24934201D81A00F824104B02
:10323000E4021B689A4210D813000E4A12689A42A0
:103240000ED3013307D1F823DB029C4203D10A4994
:10325000054808F085FB200010BDFC24E402ECE7E3
:10326000FE24E402F7E7C04600C0071100D00711B2
:1032700000E0071100F00711FFFFFF7FF0B59BB0E2
:10328000150004900391402A00D9A0E006AB5980B4
:103290001A80FFF7C2FF0400042816D9002206A9ED
:1032A000FFF768FF052810D906AB1B88AB420CD18D
:1032B000002D07D0514B2A000499C01808F048FB94
:1032C000002802D101201BB0F0BD06AB1D802000FC
:1032D0000699FFF77FFF041E7BD1069B0793FFF73C
:1032E0009CFF80235B01C618802307001B039E42BE
:1032F00001D3F826F60288235B05F31801931B68B7
:10330000013302D0019808F073FB3D49019808F0A1
:1033100027FB3B1D0293331D05938822029B520518
:103320009B181B6808935A1C3CD044219AB2009108
:10333000402A04D80320D11D814389B2009103990A
:103340001B0C8B4224D0402A22D80122300008A92D
:10335000FFF710FF021E1BD1380008A9FFF70AFF74
:103360000400042831D9009A059B9B188022520141
:10337000B218934240D288235B05C118009A09A86D
:1033800008F0CEFC1D4B009A09A9F01808F0C8FA05
:10339000009A029B9446634402931A4B029AFB18CC
:1033A0009A42BAD388235B05FC1821680198013939
:1033B00008F0D6FA200008F01BFB039A07AB5A80EE
:1033C00030000799FFF706FF0400002C03D100200E
:1033D00079E70428FBD988235B05E018069908F0F3
:1033E000BFFA0323EA1C9A4300D16BE7034B04990D
:1033F000E01808F095FA65E70424ECE704000011F2
:10340000FFFFFF7FF80F0000F7B505001400402A0A
:1034100021D8002701AE71803780FFF7FEFE042817
:1034200016D93A003100FFF7A5FE042810D93688D6
:10343000BC420BD0BD4209D0221CB44200D9321C80
:10344000064B92B2C118280008F06AFC30B2FEBDEB
:10345000C04300B2FBE703204042F8E7040000113C
:1034600037B5042204000D0001A81649FFF7CCFF70
:10347000020004280BD1019BA34208D3AB4204D025
:10348000104901A80195FFF7F9FE01203EBD0E4C41
:1034900023682000019308F0ABFA0199200001395C
:1034A000019108F05DFA80235B01E418074B9C4210
:1034B000EED10422034901A80195FFF7DFFE0020A9
:1034C000E4E7C0465555000000C007110000081190
:1034D00030B589B008F084FA10226946254808F012
:1034E000F7F9254B009A9A420ED1019B029A0F2BB5
:1034F00033D8002101240698013B08D2002900D0CE
:103500000292029B013331D10023029325E0551C26
:10351000F2D102002100EFE710341022200004A9AC
:1035200008F0D6F9029B013301D1069B0293882350
:1035300004995B05C918059B06981A03120B0491A0
:103540000592814203D02B4201D108F0E9FB019B97
:10355000013B0193019B002BDED1029B002B03D08A
:10356000049304984168084709B030BDE025014C38
:103570002D03EFE700000111504859368022F8B5BD
:10358000964C974BD200002120001C6008F068FB8D
:103590002300944A88331A60934B1A786A23002ACE
:1035A00000D01133E3620A232365904B37221B7846
:1035B0000820A3638E4B2118E361102323628D4BF7
:1035C0003B256361C823DB00A36123008C331A60B1
:1035D0002823013AE26320646364CA67043A211D28
:1035E000CA672100BC310D602100C0310860210094
:1035F000C4310B6021000635CC310D602100083D3F
:10360000C8310D602100D0310A602200D432106030
:103610002200D832136022000227E0322100176016
:103620004222DC310A6021001B3DE4310D602100A3
:10363000E83108602100EC310B6023000521F433F0
:1036400019602300F0331A602300183290331A6097
:1036500023009433186023001E3A98331A60AF2376
:10366000DB002360644BFA262363644B644DE36004
:10367000644BF031A3642300FF31FC33B600A1603A
:1036800021611E60A5627325E5656D3D6565A565D3
:1036900096255D4AAD00E264666258606766A5667D
:1036A00000270925A767E566584F594D6067200038
:1036B0002567E2673A6015279C30676007001A208B
:1036C00038602000A0300700212038602000A8309A
:1036D00007004C4838602000F83006602600642758
:1036E000A436376026005F3FAC3637602600033FC4
:1036F000B03637602600C637B4363760260000275C
:10370000B836376038269E60424E96205E64424E40
:103710005A66DE61414E9A645E62F53EFF3E9E62ED
:103720001E269A67354A8000DE661F675F67DD6583
:103730001D661862DA67BE23394A5B00E250394BD6
:10374000D838235004302250C4225200A350C6233C
:10375000E4205B00E1500433334AE1503349344BF9
:10376000D1603449800019503349E938FF38195085
:1037700032490430195032493248D161324911631B
:10378000324951631900F4310860CE2030494000BD
:1037900011603049195019002F48F83108602F493D
:1037A000D16582212E4A89005A501A002D490832CB
:1037B000D1671A002C49B432116088212B4A890044
:1037C0005A501A002A49883211602A4ADA6407F0EE
:1037D000D7FF012008F0D4FAF8BDC0460004FF1F4F
:1037E0005064FF1F206FFF1F1C44FF1F4A0AFF1F6A
:1037F0003A07000080C3C9019A020000DC050000FE
:103800006A18000050C3000088130000F009FF1F71
:10381000204E00006509FF1F68100000C409000069
:1038200040420F0010270000FC00FF1F7D1CFF1FFF
:103830000000FF1FD12CFF1F5930FF1FF12EFF1F6B
:103840003D20FF1F2D27FF1F5920FF1F0522FF1FAF
:10385000C91FFF1F5129FF1F392AFF1F9519FF1F7D
:103860005D28FF1F8125FF1F8D25FF1FC91EFF1F1C
:10387000811FFF1F411EFF1FF0B502250124614B70
:1038800091B01D700293604B604E1C70604F0393AB
:10389000336800212800FB7006F076FE280006F051
:1038A0006DFD0023984205D0FA78552A02D0332ABC
:1038B00000D09AE03360042006F0CEFF07F0D0FF7E
:1038C000FFF75CFE08F03CFA1F2201240021514B57
:1038D00010AD1A70504B1C70504B1970504B19683A
:1038E0009143163A0A431A60602219689143403A9C
:1038F0000A431A6008F0ACF808F002F9494B9847FF
:10390000C120FF21484B80001A588A431A50C52213
:10391000920098588843BF390143995098584349B9
:1039200008408021C9010143802099509958C00561
:103930000902090A0143995080213D48490108F0D4
:1039400017F9032322003B49019400933A4808F0F9
:103950007FF92C22394905A808F0E2F905AC617815
:103960002078023406F02AFDA542F8D1344C354BBC
:10397000226803201A40A023DB0213432360802324
:1039800022689B041343236022682F4B1A40802334
:103990009B03134323602D4A2D4B934200D80120F3
:1039A00007F0DEFE08F074F980232268DB0413437D
:1039B0002360029B187808F0F3F9039B1878C0B2D3
:1039C00007F006FF07F00CFF2249042007F0A0FFD4
:1039D00006F00EFF00F040F800F024FE00F0CCFEF0
:1039E00000F00CFA002011B0F0BD00932100194A3C
:1039F000042008F06DF88023DB059C62FFF768FD6A
:103A000059E7C0464A0AFF1F1C44FF1F34F000401C
:103A1000DC61FF1F480AFF1F490AFF1F680AFF1FDA
:103A2000BCF00040E1A2000000E100E0FF00FFFF69
:103A30002044FF1FA456FF1F2054FF1FC0BD0011CC
:103A400014F00040FF7FF8FFFFFF9FFF0080FF1F83
:103A5000206FFF1F3B000108002210B5110011204C
:103A600007F0DEFE10BD0000F8B500230925374F32
:103A7000374C3B62E3681120AB43E36007F0D8FFAB
:103A8000112007F09DFF112008F012F94023226851
:103A900080261343236080236268DB021343636044
:103AA000A3682C4A3343A360A36828001340A36093
:103AB0008023A2689B0113431022A360236C022180
:103AC00093432364236C0F3A1343236480235B01E5
:103AD0003B62226B204B1A402263626B1A40626386
:103AE000A26B1A40A263E26B1340E363E3681B4AD4
:103AF0001340E36006F062FC2800012106F072FD2D
:103B00008023174A9B00516C11200B43536407F02C
:103B10008FFEFD21134B144A89005A508023C72081
:103B2000E26B5B031343E363E36880001D430F4BC9
:103B3000E56019580E4A1140802212020A431A50B9
:103B4000802292051A600B4B5E63F8BD00F00040C6
:103B50003CF00040FFFFDFFFEFFFEFFFFFFF7FFFC5
:103B6000003800400000FF1F5118FF1F00E100E077
:103B7000FF00FFFF0000054070B5284C238C002B90
:103B800023D0228A002A21D1DA0023826382A382F1
:103B9000E38223836383A383E38322606260A26062
:103BA000E2601F4D1F4A6420EB8093420AD8FA223C
:103BB0000020D200934205D91B4A0A21981808F028
:103BC00007F8C0B200232872238470BD0720E11CCF
:103BD000CA7F01320240CA7705D10325201DC17F6B
:103BE00001312940C17708325200A352002321003D
:103BF0001A00088A01321B180231082AF9D1221D45
:103C0000D27F9200A350626823689B18A2689B1819
:103C1000E2689B185B099BB2C3E7C0461C61FF1FAB
:103C2000C461FF1FB70B000030F8FFFF30B503A8D9
:103C300004880B20002C0ED14968074D087849787C
:103C4000090201430A20A94205D10121200019805F
:103C5000024B1B7A137030BD192A0000C461FF1F8C
:103C6000F7B5150008AA16884A680F4F14785278DD
:103C7000120222430A24BA4214D10122DBB2019279
:103C800000962A0007F004FD041E0BD1074B1B68A9
:103C9000002B07D068782A78000210434242504136
:103CA000013098472000FEBD022900004861FF1F37
:103CB00030B5012503790400BFB02B4211D00A4969
:103CC000408807F051F828420BD0084B01A95B8DC2
:103CD0004D800B80064B00221B7A60880B7104F02C
:103CE00035F93FB030BDC0464061FF1F5040FF1F57
:103CF000C461FF1F10B50549054806F0EBFF04211C
:103D0000044A054806F0A8FF10BDC0464061FF1FE9
:103D1000FFFF0000ECBD00115040FF1F10B502482E
:103D200004F096FF10BDC046B13C001101230370A2
:103D30000B4B1A7A4270022282709A78C270DA783B
:103D40000271032242711A7982715A79C2710C226E
:103D500002729A794272DB7983720B207047C046F7
:103D6000C461FF1F022310B50370013B437005338C
:103D7000837010330371443B43712A33837144339E
:103D8000C37100230372064B04001B8843720A3080
:103D9000FFF7CCFF831D0A30C0B2E37010BDC046F0
:103DA000C461FF1F10B5142007F032FF124B14221C
:103DB0000021186007F054FF002007F0E1FE012009
:103DC00007F0D6FD022007F0B3FF032004F0E4F96A
:103DD000042006F0F9F9052003F022FC062004F087
:103DE000EFF8072001F09CFA082006F015FF0920E3
:103DF00001F076F810BDC0464C61FF1F07F0C8FD0A
:103E0000012007F0F5FC07F05BFE0000094B10B540
:103E10000400984205D0012904D12000064906F08B
:103E200059FF10BD0229FCD1013904F0CFFE002852
:103E3000F3D0F6E7FEFF00007261FF1F70B50D7A48
:103E4000100004AA2C00168810221440154220D11C
:103E5000002E20D10A78022A18D14A6851781578A4
:103E60000E4A09022943914205D00D4A914209D0D8
:103E70001C800A2404E014220A491A8007F050FF2B
:103E8000200070BD0C2208491A80F7E71C8001242D
:103E9000F6E70824F4E70B24F2E7C046F3FF00003E
:103EA000F4FF0000A842FF1FE8BE001110B5040097
:103EB0000749084806F00EFF074804F009FE0020F5
:103EC000E40704D50721054A054806F0C5FE10BDE4
:103ED0007261FF1FFFFF00000D3E001130BE001198
:103EE0009440FF1F00B50C4BBFB01A780B4902A8D5
:103EF00000F0FCFC6B4680B2D880002809D06A46EE
:103F0000074B01A91B889380064B0022188804F0F8
:103F10001DF83FB000BDC0465061FF1F5161FF1F3B
:103F2000EE40FF1FF841FF1F00B50C4BBFB01A78E1
:103F30000B4902A801F050FF6B4680B2D8800028E0
:103F400009D06A46074B01A95B8D9380064B00227E
:103F5000188803F0FBFF3FB000BDC0467A61FF1F29
:103F60007B61FF1F9440FF1FF841FF1FF7B50E0054
:103F7000377A1C0008AB11003D001A8820231D4031
:103F80001F423CD13378022B3BD173681F785B789A
:103F90001B023B431E4FBB4208D01E4FBB4214D0F6
:103FA0001D4DAB4221D00A252800FEBD002A2AD192
:103FB000142C2AD82200F06807F0B2FE174B1C70B0
:103FC000012CF1D9FFF7B0FFEEE7002A1BD1202C1E
:103FD0001BD82200F06807F0A3FE114B04211C70CF
:103FE000104B187807F064FCDEE7E3B2012400927E
:103FF00001940A00310007F04BFB0500D4E70825C7
:10400000D2E70125D0E70B25CEE70D25CCE7C0464A
:10401000F3FF0000F4FF0000022900007A61FF1F97
:104020005061FF1FFC61FF1F332310B504000370B4
:104030000A220749013007F073FE064B0F201B6868
:104040001A0AE37222731A0C1B0E6273A37310BD5B
:10405000C461FF1FEC61FF1F30B501250379040027
:10406000BFB02B4213D00B49408806F07DFE28429A
:104070000DD06A46084B02A81B889380FFF7D4FF37
:104080006B46D8800022608801A903F05FFF3FB033
:1040900030BDC0467261FF1FEE40FF1F10B50248E1
:1040A00004F0D6FD10BDC0465940001170B5160091
:1040B00004AA148805AA15784A6850781178000275
:1040C0002A4A0843801805284BD807F0E9FB031358
:1040D0001E29343F0720042C0BD80522121BAA42AC
:1040E00000D92A0022491A803000091907F018FE69
:1040F000002070BD0720112CFBD81222121BAA42EF
:1041000000D92A001B491A80EEE707200E2CF0D8B0
:104110000F22121BAA4200D92A0017491A80E3E78E
:104120000720032CE5D80422121BAA4200D92A003A
:1041300012491A80D8E70720032CDAD80422121B70
:10414000AA4200D92A000E491A80CDE70720032C85
:10415000CFD80422121BAA4200D92A0009491A808A
:10416000C2E700220A201A80C3E7C046DCD5FFFF61
:104170007BBE00119861FF1F6BBE001166BE00116F
:1041800061BE00115CBE001110B50D21024A03484A
:1041900006F062FD10BDC04650BE00110441FF1F75
:1041A00013B5104C0423217C01AA00F0ADF90028BE
:1041B00015D16B469A88236852BA92B2534322892A
:1041C00009491B0C9B184B806B46DA88636852BA0E
:1041D00092B2534362891B0C9B188B8016BD012041
:1041E000FCE7C046AC61FF1FC461FF1F13B5124C52
:1041F00006236A46217C00F087F9002819D16B4616
:104200001988236849BA89B24B4321890B4A1B0C90
:104210005B1853806B46D97803335B781B020B43E2
:104220005BBA61689BB24B4361891B0C5B1893803E
:1042300016BD0120FCE7C046AC61FF1FC461FF1F33
:1042400037B5174C07236A46217C00F05DF900283A
:1042500024D16B461B787F2B20D86B46DD78F0236A
:104260002A041B031A406B469B880E495BBA9BB21B
:104270001A4323682D09534322891B0C9B184B803A
:104280006B465A789B7812031B011A4363682A43D2
:10429000534362891B0C9B188B803EBD0120FCE7B9
:1042A000AC61FF1FC461FF1F7FB50226154C0022C1
:1042B000217C03AB0096050000F0F8F8002802D03E
:1042C000012004B070BD0E23217C0122280000963D
:1042D0006B4400F0EBF80028F2D16B469A89236812
:1042E000D2BA5343228908491B149B184B806B4652
:1042F000DA89636852BA92B2534362891B0C9B18E5
:104300008B80DEE7AC61FF1FC461FF1F70B5184CE6
:10431000237C002B0FD0382B0ED1164D280000F037
:1043200073F8CC23AC222800217C9B0100F027F9F4
:10433000280000F0A7F870BDE3890F4A934209D125
:104340000C4D280000F060F800222800217C00F0CD
:1043500005F9EDE7094A9342EDD1064D280000F03A
:1043600053F890222800217C920100F026F9DFE723
:10437000AC61FF1FDC41FF1F8305000083200000AC
:1043800070B5144C237C002B1FD06369002B1CD00C
:10439000114D280000F038F86369280098470400A0
:1043A000280000F06FF8002C10D10C4B0422995E0D
:1043B000002905DA9C801A8801321A80200070BD1D
:1043C000074A9142F7DD9A80F5E70124FEF790FE57
:1043D000F4E7C046AC61FF1FDC41FF1FC461FF1F53
:1043E0000F27000010B58024064AA4001168436B13
:1043F000234205D113685B1A032BF8D9012010BDA5
:104400000020FCE76008FF1F70B5C17905000C00B3
:10441000631E9C411A4BE402E41849000460C9B2CF
:10442000007906F015F9E979687949000131C9B2D6
:1044300006F00EF9E8790930C0B207F039FC002324
:10444000E36661332360AA795B3B002A0ED02268C1
:104450009A43023B134323600A23E3610733236239
:1044600000232363A3630133E36370BD22689A438F
:10447000022313432360462363610633A361EFE7FE
:104480000050004070B5002504000368DD66C07967
:104490000930C0B207F0CCFA2900207906F074F890
:1044A0002900607906F070F870BD0000F8B51E00B4
:1044B00006AB1D78002304681700E366616007F00F
:1044C0008FFA01238022E3662B0027615200013B13
:1044D00008D207F0C5FA08200A4A1168002D03D156
:1044E0002800F8BD2261F2E7236F034203D023695D
:1044F000013D3370013613685B1A032BEED9012599
:10450000EEE7C0466008FF1F70B51C000023056879
:104510001600EB66696007F063FA01238022EB6600
:1045200023005200013B08D207F09AFA08200A4AF9
:104530001168002C03D1200070BD2A61F2E72B6FB7
:10454000034203D02B69013C3370013613685B1AB8
:10455000032BEED90124EEE76008FF1F002370B59E
:1045600004681500E366616007F03AFA0123E36628
:10457000256107F075FA2000FFF734FF70BD70B5B4
:104580001D00002304681600E366616007F028FA46
:104590000123E36626610F33626B1A42FCD02B0ABB
:1045A00023611023626B1A42FCD0EDB2256107F043
:1045B00057FA2000FFF716FF70BD002370B504689E
:1045C0001500E366616007F00BFA0123E3662B0A2E
:1045D00023611023626B1A42FCD0EDB2256107F013
:1045E0003FFA2000FFF7FEFE70BD70B51E000023ED
:1045F00005681400EB66696007F0F2F90123A6195B
:10460000EB660F33B44205D107F02AFA2800FFF712
:10461000E9FE70BD21782961696B1942FCD0013433
:10462000F0E7000010B5084CE368002B08D18022A9
:10463000064B52021B689B186360054B1B68236086
:1046400007F04EF9A06010BDEC61FF1FC8F00040FC
:10465000CCF0004070B5184A936A916A9942FBD138
:1046600016498A689A421FD39A1A8B60144B012606
:10467000186893B2D202D20E4343424300204C68E2
:104680001B0A1B1912029B180E4C0A684B60551C22
:10469000A3420CD8002801D04B600A600A4A13607C
:1046A00008680A4B186070BD581E821ADDE7084A78
:1046B00030009B182A00EAE700F00040EC61FF1F81
:1046C000140AFF1F40420F00C8F00040CCF0004029
:1046D000C0BDF0FF70B51F4C23793F2B01D93F239C
:1046E00023711D4B22791A701878C0B207F018FA9E
:1046F00018231A491A4A0B801A4913800B805380D9
:10470000A379194980200B800C21938001334B43FE
:10471000164D191C0001834200D9011C2980D1804B
:104720006379002B11D101336371237A012B01D8F6
:10473000022323726279237A0D4853430A21584396
:1047400007F046FA0B4D286070BDA02BEDD9A023D1
:10475000EAE7C046E061FF1F480AFF1FF641FF1F5E
:10476000C843FF1FF441FF1FF241FF1FF041FF1F2D
:1047700071020000D061FF1FF8B520210020FEF774
:104780006FFE114C011E114D09D10C22104BC1CBF3
:10479000C1C4280007F064FAFFF79CFFF8BD0C22A3
:1047A00020000C49FEF730FE0C2802D0084B43CB0A
:1047B00043C40C2228000849FEF726FE0C28EBD043
:1047C0000C220021E5E7C046E061FF1FAC61FF1F3E
:1047D000DCBE0011FC0C0000F50C0000F0B51D4C17
:1047E0008022A5440400882069465201400507F054
:1047F000DFF9902212016A441300200032C832C34C
:1048000016C816C38023144C144FA6689B03334369
:10481000A3603B6006F0C4FF8823A0685B05C01856
:1048200007F0E6F80025882329008022A0685B05B0
:10483000C01840196944520007F072F8802301350E
:10484000FF355B019D42EED1A6603E60044B9D4466
:10485000F0BDC046FCEFFFFF3843FF1F9808FF1F65
:1048600004100000F0B5040087B0002825D0684689
:1048700007F03EF81B4C022806D1062269462000AC
:1048800007F066F8002816D06946002301250F2698
:104890002F00E25C013310091030874038002F00F0
:1048A000324097403A0002434A610439062BEFD167
:1048B0006846FFF793FF07B0F0BD182269460A4823
:1048C00007F076F96A46A300D358013305D01822C1
:1048D000FF21684607F0C4F9EAE70134062CF1D15C
:1048E000E9E7C0466509FF1F00090011F0B5002582
:1048F00004000E0085B0AA4200D186E04B1C087867
:1049000001934B788978377909021943F3783F0688
:104910001B040B431F43039720706570252800D1AB
:1049200096E033D8112813D807F032FA690028012D
:10493000280128012801AA00B800B1002801280197
:10494000280128012801280128012801020122014B
:10495000232800D1DBE0DB2800D031E1042A00D895
:10496000ACE01025052A05D0551F2A003800711D1E
:1049700007F0D6F905223100200007F0D1F92A000E
:104980003900601D07F0CCF905353EE0562859D0B6
:1049900010D8332800D19DE0552839D02628DAD107
:1049A0009D4B2900132218001D0007F059F9FEF74E
:1049B0009FFB5CE0712800D177E0722800D180E095
:1049C000602800D18BE0DC28C5D1022A00D875E030
:1049D0007378BFB26370B378A370032A05D0033A2B
:1049E000390092B2F01CFEF749FC10223900E01C9D
:1049F000FEF70AFDC51C002807DA60705CE00C2297
:104A00002000864907F08CF90C25280005B0F0BD80
:104A1000013A834D0C2A13D8002A0AD028000199A4
:104A200007F07EF9FFF756FE0C2228007D49FEF7BD
:104A300025FC29000C22601C07F072F90D25E4E723
:104A40000C22EBE7764D784B2A0043CB43C2E9E7D3
:104A5000013A714D0C2A11D8002A08D0019928007A
:104A600007F05EF90C2228007049FEF707FC2900C8
:104A70001322601C07F054F91425C6E70C22EDE759
:104A800006226B49601C07F04BF90625BDE7122290
:104A90006849601C07F044F91325B6E70822664907
:104AA000601C07F03DF90925AFE77178F02905D8BA
:104AB000624B188801F0ECFD0225A6E7FF23637026
:104AC000FAE75F4B012A03D072789A706270F3E7BD
:104AD0009B78F4E72000FFF7A7FA050095E7013A75
:104AE000574B584D082A0DD8002A0DD00121280017
:104AF0005970019907F014F901F086F8082229008D
:104B0000601CCEE70822F1E700225A70F6E7042A7B
:104B100004D94D4D2F6006F0E3FEA860FFF79AFD23
:104B20000422039003A9601C07F0FAF805256CE73E
:104B3000464D062A15D906222800019906F008FFDD
:104B400000280ED006220199280007F0E9F8062275
:104B50003F492800FEF792FB0123394A91780B4325
:104B6000937029000622601C07F0DAF807254CE74D
:104B7000012AA3D07078FFF775FE9DE7012800D0C9
:104B8000E9E6931E334F132B06D87378002B0BD115
:104B900000F014F900F04AF92F4B39001D78601C21
:104BA0006A1E07F0BDF830E7551E2A00019938004B
:104BB00007F0B6F838002949AAB2FEF75FFBE9E72B
:104BC000DA281DD1042A00D878E7082A15D9B37944
:104BD00072791B021343F27912041A43337A1B06CB
:104BE00013433B603B68052231002000039307F02C
:104BF00097F80422601D03A953E7FE236370F1E7D1
:104C0000DE2800D05AE7511E012A01D10025FCE61A
:104C1000019800F0DFFFF9E7AC61FF1FE8BE00116B
:104C2000E061FF1FFC0C0000DCBE0011F50C000071
:104C3000B861FF1F9861FF1F3C43FF1FF841FF1F32
:104C4000DC61FF1F9542FF1FEC61FF1F6509FF1F1D
:104C5000ADAC0000DD63FF1FDB63FF1FAEDE0000B5
:104C600070477047020010B5094B0A32094C92B2E6
:104C7000DA815A8298811882207802F06FFB042230
:104C8000054B012120781A7006F012FE10BDC046B7
:104C9000C642FF1F2664FF1F2564FF1F013870B541
:104CA000042809D806F0FCFD030928081200234B4C
:104CB0000221187806F0FCFD70BD204B0821187801
:104CC00006F0EEFF00221E4B1A72F5E78022002448
:104CD0001B4B1A4D52001A8108211A682878DC7281
:104CE00006F09EFF2100287806F052FF012000F018
:104CF00077FE00F089FFDFE7104B0821187806F0F7
:104D0000CFFF1048FFF72EF80F4B104A9B79002079
:104D100093800F4A13808022094B5200D8721A8167
:104D200000F05EFE00F070FF0A4B9B78002BC3D0B2
:104D3000094A136006F0ECFFBEE7C046FC61FF1FA6
:104D4000D061FF1F0142FF1FE061FF1FC843FF1F2B
:104D5000F241FF1FDC61FF1F34F0004010B5012954
:104D60000BD1022809D1054B1B78002B05D0262238
:104D7000034B04485A72FFF775FF10BDFE63FF1F17
:104D8000D061FF1FC40900000300F0B50A4D8E1862
:104D9000B14202D152008018F0BD0C782F6824096E
:104DA0003C5D0F271C700C7801313C402F683C5D46
:104DB0005C700233ECE7C046EC41FF1F0E22124B41
:104DC00010B51A700D23114C11492370093A043B98
:104DD0001048637006F0A4FF2D2301220E490F48EE
:104DE000E371FFF7D1FF01220D49FFF7CDFF01224B
:104DF0000C49FFF7C9FF030000200B49020018709F
:104E0000FEF73CFA10BDC046FA63FF1FDB63FF1FCD
:104E10007BBE0011DD63FF1F6709FF1FE363FF1FF8
:104E20006609FF1F6509FF1FAEDE000070B5134C59
:104E3000142220001249FEF7E7FA431E114D132BEE
:104E400019D8AB78002B16D0431C2B7009236B703C
:104E500000230019037028780B4B01302900C0B2E1
:104E6000187006F0A5FF297822000139C9B2002088
:104E700005F010FE70BDFFF7A1FFECE7DD63FF1F3B
:104E8000AEDE0000DB63FF1FFA63FF1F10B5114B9E
:104E90001A781870002A0ED000280BD10E4B1A7801
:104EA000062A07D85423D340DB0703D50B4B1878C9
:104EB00002F054FA10BD0028FCD0074B1B78012BE0
:104EC00002D0033B022BF5D8044B0121187806F0E1
:104ED000EFFCEFE7FE63FF1F2564FF1F2664FF1F43
:104EE00070B54A4E4A4A4B493070022005F05EFCCC
:104EF00000F00EFFFEF7FCF806F02AFE03224649FA
:104F00004648FFF741FF2D24030004221C7044494A
:104F10000130FFF739FF30230470424D424C43709B
:104F200083702E3B062220004049EB87FEF76CFA87
:104F3000062813D0200006F0DBFC022809D003214C
:104F4000200006F035FD8D23E3706E3B237119338D
:104F50006371062220003549FEF790F9344B1B6837
:104F6000FC335C64FFF762FF0020FFF78FFF314CDA
:104F7000314A0121314B1278207802F0B1F9304AE0
:104F8000304B12780021207802F0AAF901222E4B32
:104F90001A702E4BDB78552B31D12D4B3B325A7288
:104FA0002C4B2D4AAB81EA812B826A8220213078FA
:104FB00006F0A6FE0120404205F0B8FD0120404267
:104FC00005F054FEFFF7E0F8FEF794FE00F0B2FCA7
:104FD00001204042FEF76AFF012006F0A9FCF02004
:104FE00001F03AFB0121307806F062FC307802F0E3
:104FF00011FB1A4806F07CFEFEF736FD70BD6422F8
:10500000174B5B7953431A000A32CBE7FC61FF1F51
:10501000614C00115D4D00113C43FF1F9861FF1F63
:10502000B861FF1FC642FF1F6509FF1FADAC00003E
:105030005064FF1F2664FF1F2042FF1F0142FF1F15
:10504000FA63FF1FDB63FF1FCC63FF1FDC61FF1FE1
:10505000D061FF1FC4090000CE090000FE61FF1FE0
:10506000E061FF1FF8B50A0020230D001A40194225
:1050700063D05E4B1B78002B5CD0FFF7EBFA5C4BE8
:105080005C4C5D4E99686268737A8A1ADB039A42B7
:1050900002D36160FEF7E8FC327A217A531EDBB25C
:1050A000994205D1FFF732F9002000F0E9FD15E043
:1050B0009142F9D300272772FFF762F9A37ABB4226
:1050C00002D0A772FEF758FD012000F0D9FD4B4F2A
:1050D0003800FEF747FE390006F0AAFD637A002B80
:1050E00025D0013BDBB26372002B20D1444BDB782F
:1050F000552B01D106F00CFEE37A002B12D00023D1
:10510000A27AE3729A4202D0A372FEF735FD3D4ABD
:105110003A4F1388380001331380FEF723FE39001D
:1051200006F086FD642370795843FFF79BFD237AD0
:105130000133237220206840F8BD0BB2002B0ADA3D
:10514000314B187806F044FC002801D006F008FD29
:1051500080200002EFE70224214206D0254B0120E7
:105160001A72FFF793FE2000E5E70B071ED5FFF745
:1051700071FA1F4B1F49204C98684A68637A821A5B
:10518000DB039A4202D34860FEF76EFCFFF7F8F8A3
:10519000FFF7BCF8012000F073FD00F0E5FB236889
:1051A000DB0701D5FEF77AFF0820C4E7CB0609D557
:1051B000FEF7E2FC0D4B1B78002B01D1FEF7AEFD94
:1051C0001020B8E70124214207D0104800F06CF805
:1051D00006F0B6FC00F034FDC5E7042408002040CA
:1051E0002142A9D0FEF77EFEBDE7C046FE63FF1F49
:1051F000EC61FF1FD061FF1FE061FF1F0142FF1F35
:10520000DC61FF1FC461FF1FFC61FF1FE441FF1F42
:10521000F0B51B4B1B4F1B883A8804001A4E1B4DE0
:1052200085B09A420DD832889A420AD3184B1A8810
:105230002B889A4205D1174A174B12881B889A422D
:105240001BD0052001F05EFA3B8802AA1380338848
:10525000019053802B88114D93800F4B02A91B881E
:10526000D3800F4B2A78188802F07AFF0D4B082163
:105270002878019A1C7006F0A3FC05B0F0BDC0466A
:10528000CA63FF1FF641FF1FF441FF1FF241FF1FDA
:10529000C863FF1FC663FF1FF041FF1F2664FF1F87
:1052A000F841FF1FC463FF1F13B50C4B1C78002C83
:1052B00011D1002801D00A4B18600A4A0A4B117814
:1052C0000A4A10780A4A01920A4A0092002205F01E
:1052D000D9FA200016BD1124FBE7C0462564FF1F44
:1052E000C063FF1F2464FF1F1464FF1F2664FF1F99
:1052F0000064FF1F0464FF1F10B5064B12201B78CB
:10530000052B06D1044B13221988044B187801F0A1
:10531000D5FB10BD2564FF1FF841FF1F2664FF1F4A
:1053200010B500240122114B52421870104B1C7012
:10533000104B1A8002F06EF904220F4B21001A70F4
:105340000E480C3206F094FB102221000C4806F0A7
:105350008FFB07220B4B1C600B4B1C700B4B1C7004
:105360000B4B1A700B4B1C7010BDC0462664FF1F00
:105370002564FF1FF841FF1F2464FF1F1464FF1FF3
:105380000464FF1F0064FF1FDA63FF1FD963FF1F60
:10539000FA41FF1FD863FF1FF8B5174C06002578A8
:1053A00006A814240078052D23D1B41F134FA5B2ED
:1053B0001824BD421DD88D1FADB2BD4219D8FA25A3
:1053C0006D00AA4215D21D000D4F0A3DADB2BD427F
:1053D0000FD80C4C26800C4C21800C4900240A80EC
:1053E0000B4A1380FFF714FF0A4B0421187806F0CC
:1053F00057FC2000F8BDC0462564FF1F790C000053
:10540000750C0000F641FF1FF441FF1FF241FF1F22
:10541000F041FF1F2664FF1FF0B50BB20D0089B0ED
:10542000002B00DB70E1A44E307806F0D1FA041EA8
:1054300050D00378A22B00D122E1D02B1AD0912B8F
:1054400045D143780E2B42D19C4B82889A423ED163
:105450009B4A83681278052A39D1032018567F2881
:1054600035D0984B1B68002B31D05B68002B2ED0B9
:1054700098472CE08078072829D806F011FA0428EC
:10548000183F3F74A8D86378002B0CD101218C4BB6
:1054900019708D4B1A78002A5BD08C4B307801F054
:1054A0001FFF002855D00722854B1A7051E0617804
:1054B0000029F8D1E378002B11D0854A854B12786A
:1054C000307801F00DFF60706378002BEBD1200085
:1054D00006F046FB80200002684009B0F0BD784B22
:1054E0001B78022BF3D00121307806F091FA0028C6
:1054F000EAD10121307806F0DBF9E5E76378002B8B
:10550000D1D16F4F032807D13B78052B02D101334E
:105510003B701EE00223FBE76F4B1A886F4B029330
:10552000002A0BD01B78002B03D00121307806F025
:1055300047FB3B78062B04D1013BE9E7029B1A703D
:10554000F7E7042B41D10121029B3078197006F056
:10555000AFF95C4B1B68002BB9D01B68002BB6D091
:10556000574A107884E76378554F002B27D10622DD
:10557000211D5B4806F0D4FB62895A4B5A491A80B8
:10558000A2895A4B1A80E3890B800521397058494A
:105590000A80584A1380228A574B1A80574B1B782F
:1055A000012B09D11F2001F0ADF8FA2292004243ED
:1055B0000421307806F004FB0022484B75E7312BBC
:1055C00000D070E70022454B1A700323A0E70622A3
:1055D0000021434806F04CFA0023454A0421138079
:1055E000444A30781380444A138006F059FB08215E
:1055F000307806F055FBA379083B5A425341304AB4
:1056000003331370304B1B78002B06D0334B3078AC
:105610001A78002A06D001F0A1FE0122314B524235
:105620001A8096E70121197006F042F9F5E7082182
:10563000307806F035FB6378002B00D047E72C4B21
:105640002D4F0293E388029A04211380294B30786E
:1056500003932389039A138063893B8006F0D8F96A
:10566000002800D033E7264B1B68002B00D12EE723
:10567000039902983A88098800881B68984726E7AA
:105680004379132B00D022E70389012B0AD11D4B4C
:105690001B78022B06D10821307806F001FBFFF7BA
:1056A0002BFE14E7052001F02DF8082102003078C8
:1056B00006F086FA0BE7C0462664FF1F05140000BB
:1056C0002564FF1FC063FF1F2042FF1F0142FF1F11
:1056D000FA63FF1FDB63FF1FFC63FF1FFE63FF1FF7
:1056E000CD63FF1FF841FF1FD463FF1FD663FF1F69
:1056F000CA63FF1FC863FF1FC663FF1FCC63FF1F82
:10570000BC63FF1FC463FF1F8020C001014200D0A3
:10571000E2E6CB0731D5324B1B78002B1DD0314E42
:1057200005AC3378052B1AD1023B23702E4B210098
:105730001B7823722D4B1B7863722D4B187801F068
:1057400073FD002809D007202A4B30701B68002BFE
:1057500003D01B68002B00D098470120BCE60E2028
:10576000254B06221B7825492370254B1B78637037
:1057700002ABC01806F0D4FAD8E70223080018409C
:10578000194209D0174B1B78052B03D11D4B1888E4
:1057900006F036F802209FE60424214203D0FFF7EA
:1057A00037FD200098E6082308001840194200D170
:1057B00093E6154B1C78012C03D0022C0DD0082049
:1057C0008AE6124B124A134913481B88128809882B
:1057D00000880094FFF7E0FDF1E7FFF78DFDEEE7AD
:1057E000FE63FF1F2564FF1FFA41FF1FD863FF1FE1
:1057F0002664FF1FC063FF1FDA63FF1FFB41FF1F0B
:10580000D963FF1FF841FF1FC463FF1FF041FF1F53
:10581000F241FF1FF441FF1FF641FF1F10B502A820
:1058200004880B20002C10D14968087849780902B7
:1058300001430C48814209D1022119800A4B598841
:105840001170DB7800205BB2537010BD074C0A204A
:10585000A142FAD102211980034B998811705B791A
:10586000F0E7C0466E2A0000C461FF1F6F2A0000E7
:10587000F7B5150008AA16884A680F4F14785278B1
:10588000120222430A24BA4214D10122DBB201924D
:1058900000962A0005F0FCFE041E0BD1074B1B6886
:1058A000002B07D068782A7800021043424250410A
:1058B000013098472000FEBD022900003864FF1F18
:1058C00030B5012503790400BFB02B4225D014491F
:1058D000408805F049FA28420CD0124B01A95B8D93
:1058E00000220B8002234B800F4B5B888B806088EB
:1058F00002F02CFB0D49608805F036FAC0070CD584
:105900000B4B01A91B8800220B8002234B80064B06
:105910009B888B80608802F019FB3FB030BDC04689
:105920003064FF1F2442FF1FC461FF1F2864FF1F54
:105930007E42FF1F10B5074C0749200005F0CAF949
:105940002000064905F0C6F90721054A054805F07B
:1059500083F910BDFFFF00003064FF1F2864FF1FA4
:1059600008BF00112442FF1F10B5024803F070F970
:1059700010BDC046C1580011082110B50E240A4AB6
:10598000C307DB170B405179A1430B43537102232B
:10599000184202D051790B4353710423184202D0AC
:1059A00051790B43537110BD9542FF1F0A2110B569
:1059B0000F240A4AC307DB170B401178A1430B439E
:1059C0001370830703D5062311780B431370400728
:1059D00003D5012311780B43137010BD9542FF1FAF
:1059E00010B5054B102419780A00A243002801D0F5
:1059F00022000A431A7010BD9542FF1F662110B5A0
:105A00002024134BDA788A431979DA70A1432419D8
:105A10000C431C71542812D96020014319710421D0
:105A20000A43DA700222D9780A43DA702022D97840
:105A30000A43DA704022D9780A43DA7007E0442832
:105A4000EDD83428EED82428F0D81428F2D810BD88
:105A50009542FF1FF8B50E23384C05006279267970
:105A60001A4011339E43364B62712671984204DD11
:105A70006E23E3716C3BA371F8BD324B984203DA9D
:105A80001A23E3711C33F6E700232F49A371E37156
:105A900083B259182D4889B2814224D9681D0A2140
:105AA00000B206F095F82A4B00B29D4244DC050096
:105AB0006421280006F08CF80A2100B206F0C0F834
:105AC000244F09B2E2797B5C1343E3710A21280079
:105AD00006F07EF80A2100B206F0B2F81D4F09B2B6
:105AE0007B5CA2790EE001210A436271002D1CDA71
:105AF0005B421DB20423A371A379632DD8DCFA2283
:105B0000092DE3DC1343A3710A21280006F098F85D
:105B10000F22114F09B27B5C1A4016431F22934398
:105B20006279267113436371A6E7FA239B009D42B5
:105B3000E2DB0123E371BBE70500FAE79542FF1FB3
:105B40001B4E00001DFCFFFFCB070000960F00005E
:105B50000A27000052BF001142BF001170B51B4D53
:105B600004002B7900290DD0802213432B71632C64
:105B70000BDD76236A7813436B704023AA781343B6
:105B8000AB7070BD7F221340F0E72300093306DAC3
:105B900058236A7813436B70AA786C23EFE70C4E96
:105BA000002C0ADA2023644224B26B700A21200000
:105BB00006F046F809B2735CE2E7092CF6DD0A212B
:105BC000200006F005F800B2335CEEE79542FF1FB7
:105BD00032BF0011F8B50A4F05003B780E00002BCC
:105BE0000CD0084C2000FEF70FFC33002A002000E8
:105BF0003978FEF7FAFC2000FEF744FCF8BDC046F9
:105C00004564FF1FA042FF1F70B50A4E0A4D0822CF
:105C10003100280005F09CFE002809D0074C310017
:105C20000822280006F07CF809212000FFF7D2FFA7
:105C300070BDC0469542FF1F3D64FF1F3C64FF1FBF
:105C4000102110B50D4B1A780A401A70DA785631C7
:105C50000A40DA70602219791140223ADA71083A62
:105C60009A71AA325A71DF3A0A431A716B225A703A
:105C70000C3A9A70FFF7C8FF10BDC0469542FF1F4F
:105C800010B5002832D01E4C0223E05E1D4B1B686D
:105C90005B062CD509233221584305F099FF41308A
:105CA000FF3000B2FFF7D6FE0520FFF765FE0422A5
:105CB000A35E154A6320934205DC32331800642149
:105CC00005F086FF00B20121FFF748FF207AFFF7B9
:105CD00095FE0020FFF76AFE0C4B1878053843420A
:105CE0005841C0B2FFF77CFEFFF78EFF10BD0A21BE
:105CF000053005F06DFF00B2FFF7ACFE0320D4E7DE
:105D0000C461FF1FE061FF1FDD2600002564FF1F47
:105D100070B500250A4C2000A571FEF775FB102315
:105D20003E212000074AFEF760FCA84200D13E3524
:105D3000054B20001D70FEF7A5FB0123A37170BD6C
:105D4000A042FF1F22BF00114564FF1F0200F0B5F3
:105D500001270A480A4E51188B1A002B00DCF0BDAF
:105D6000082415784308684038404000805B013CB7
:105D700058406D08002CF5D10132EDE7FFFF00001F
:105D800062BF0011F0B500250F269D4200DBF0BD7B
:105D90004C5D070944403440A400A05801357840C8
:105DA000F3E70000F0B589B06A460D000B000F273D
:105DB000110010351C780133260024093E4016706E
:105DC00054700232AB42F5D12023024AFFF7DAFFCA
:105DD00009B0F0BD68BF0011F0B54E780B7889B0FE
:105DE00036020C00170001901E43012A61D9954B21
:105DF0009E4200D877E001339E421CD1062A17D17B
:105E0000CA788B7812021A430B791B0413434A7920
:105E100012061A438C4B5A6100221A705A808B4A20
:105E20005A608B4A9A608B4ADA60002009B0F0BD54
:105E300088225205EEE7884B9E423CD182498B78FE
:105E4000002B00D0F6E00C2A31D10F22A378934327
:105E5000E278120213432279120413436279120684
:105E600013434B60E279A07912020243207A0004C6
:105E70001043627A12060243CA60E27AA07A1202E2
:105E8000024376484A81834208D804236E4914228B
:105E900001980B7005F044FF1420C7E71201D218D7
:105EA00089235B059A42F0D801238B70BDE7022A53
:105EB000FAD00523EAE76A4A01239642E6D1FFF7C2
:105EC0001BFA052F0CD9E378A2781B021343227921
:105ED00012041A4363791B061343624A0393136047
:105EE00005F016FFA1E7584D2B78002B9DD1AB781C
:105EF000002B00D1A0E02B8901339BB20093B34269
:105F000000D091E0132AD4D9CF7C8B7C3F021221A0
:105F100020001F43FFF71AFF874200D08EE0002EBB
:105F20003DD1E378A2781B0213432279E968120479
:105F30001A4363791B06134303930A228B4212D13F
:105F4000FF23A370E370237163716B89002B09D168
:105F5000E37B227C1B0212041343A27B13431B0925
:105F600001336B8100226B89002B8ED0002A67D110
:105F7000686837013818000B6B690003039098427A
:105F800005D9686105F034FDEB780133EB70686882
:105F90001022A11C381805F0C3FC2E8145E76F893B
:105FA000009A7B1E9BB293423AD1E278A378120208
:105FB0001A43237905A81B04134362796C681206FF
:105FC0001A43EB6800920392211D0C22049305F002
:105FD000A7FE0120260004A940421036FFF7E2FE8A
:105FE000013F012F17D1009A0B232861824200D074
:105FF0004CE704221C49200005F092FC042203A96E
:10600000686805F0D5FDE968039AFF23914200D145
:106010003CE7F73B3AE73100FFF7C4FE1036DFE715
:106020000923B742A4D831E7009BB34200D9FCE66C
:1060300007232BE7022329E7032327E7062325E786
:106040000A2323E7FFFE0000A842FF1F0000011102
:10605000FFFF00005048593601FF0000FFFF00110C
:1060600002FF000034F00040B442FF1F10B5034CA3
:106070000B000122210000F06BFA10BD2D6200110F
:106080000B8870B506000D000224162B11D92B00C9
:106090000322094900F05CFA041E0AD1074B2A8842
:1060A0001B88191C934200D9111C300089B200F0E2
:1060B000EFFA200070BDC046596200115664FF1F00
:1060C00010B54A780400013A0B000220012A07D8D3
:1060D0000A78002A04D005222000024900F038FA8C
:1060E00010BDC046876200110A7810B50B0004008D
:1060F0000220002A04D007222000024900F028FADA
:1061000010BDC046336300110A7810B50B000400BF
:106110000220002A04D009222000024900F018FAC7
:1061200010BDC0469963001110B5034C0B000B2243
:10613000210000F00DFA10BDC963001110B5034C29
:106140000B000D22210000F003FA10BD3B6400118A
:1061500010B5034C0B000F22210000F0F9F910BD1F
:10616000956400110A7810B50B0004000220002A83
:1061700004D011222000024900F0EAF910BDC04607
:10618000A5640011002310B51322190000F0E0F9F6
:1061900010BD000010B5034C0B001722210000F0C9
:1061A000D7F910BDF7640011002310B519221900AA
:1061B00000F0CEF910BD000010B5034C0B001B22FF
:1061C000210000F0C5F910BD31650011F7B58489D3
:1061D0000D0006000121002C22D000238268D35636
:1061E0001778002B1EDA0C2C1AD90C3CA4B2131908
:1061F00040880093230002F086FE431E9841013040
:106200007B06DB0F6B703F23013C1F40A4B228705C
:10621000AF70AC80002C07D0B3680133AB600021B5
:106220000800FEBD0020EBE7AC60F8E70B780370D8
:106230004B8843704B881B0A83700B79C370042012
:1062400070470420022B06D10020537811781B02DE
:10625000009A0B43138070470B8803700B881B0A4E
:106260004370022070470420009983420AD153787A
:1062700010781B0203430B80D37890781B020343F2
:1062800000204B807047F8B50D004B7801240021A9
:10629000461C03702B788B4201D82000F8BD6B7828
:1062A000B01C4F1C012B10D1890069184B880222A9
:1062B00033704B88B9001B0A7370691805F058FADF
:1062C00004360434A4B2F9B2E4E7122359436B183C
:1062D0005A88043132705B8810221B0A7370691867
:1062E00005F046FA12361234ECE770B5049D14003E
:1062F0001E00052B01D8042070BD637812781B02A4
:1063000013432B80E378A2781B02134302226B8095
:106310002A71211D681D063E05F02AFAB2B22A81B3
:10632000E92AE8D82800A11D0A3005F021FA00204A
:10633000E2E7002310B50A789A4201D8900010BD18
:106340009A008A185488013304705488DBB2240AF6
:106350004470948884709288120AC2700430EAE70C
:1063600010B51100029C062B04D004201022142B1F
:1063700001D010BD022222714B7808781B02034322
:106380002380CB7888781B02034363800431601D2F
:1063900005F0EEF90020ECE710B50C788B780431AD
:1063A0005C43E4B203702200013005F0E1F9601CA7
:1063B00010BD0420022B06D10020537811781B0257
:1063C000009A0B431380704710B50C000A88023105
:1063D00005F0CEF9208810BD70B504000D000498BA
:1063E0001100012B01D8042070BD167852781202DA
:1063F000324302800200F13255701470E125002C06
:1064000000D10C35023B9AB24280AA42EBD802314D
:10641000043005F0ADF90020E6E70420009983423E
:106420000AD1537810781B0203430B80D3789078FD
:106430001B02034300204B80704710B50C000A88F4
:10644000023105F095F9208810BD000070B50121DA
:106450001E000420049C0E400B4218D1CB40DDB23C
:106460008D4214D90A49DBB2098899420FD323001F
:10647000EE331D703300580011184978165C09027C
:10648000314301332152D9B28D42F4D8002070BD7E
:10649000C042FF1F10B50C000A88023105F068F9F0
:1064A000208810BD10B50C788B7804315C43E4B2C1
:1064B00003702200013005F05BF9601C10BD10B5BF
:1064C00011000298032B01D8042010BD14785278D3
:1064D000043B120222430280CA788C7812022243C3
:1064E00042809AB28280EB2AEED80431063005F061
:1064F0003FF90020E9E710B50C000B8803700B880A
:106500001B0A43704B8883704B881B0AC3708A88B0
:106510000430063105F02CF9A088043080B210BD9B
:106520000420012B03D100201378009A13707047C8
:1065300010B50C000B8803700B881B0A43704A8847
:106540000230043105F014F96088023080B210BDC9
:10655000F0B589B003931E4B029242000700D05A57
:10656000019102F020F81325061E2DD0029B012474
:106570000370019B002B04D0001903999847001960
:1065800084B26B461B7A5BB2002B0FDA1021380005
:1065900002F01CFB1925002813D130003219E1B29A
:1065A00002F066FC051E0CD10C34A4B2042304AA2C
:1065B000380005A993800696948101F0AFFD051E71
:1065C00002D0300005F014FB280009B0F0BDC04631
:1065D0005464FF1F70B505000C0000280CD000208B
:1065E000814209D010222000044905F0C1F80120A1
:1065F0002B7823736B78637370BDC046A8BF0011FE
:10660000F0B506000D0017001C0085B002291BD054
:106610000020102907D1022B07D0102B03D115E041
:106620000020102C08D005B0F0BD69463800FFF7F7
:10663000D1FF2A0069460BE069463000FFF7CAFF28
:1066400022006946380004E0022BE9D12A00390013
:10665000300005F015F9E6E7031CF02800D9F02317
:10666000032008499AB2013A0B80D3170340064928
:106670009B189B100B80D30F04499B185B100B8059
:106680007047C046C442FF1FC242FF1FC042FF1FE7
:10669000034B1B888B4202D3024B4000C152704710
:1066A000C442FF1F5464FF1F014B4000185A70473B
:1066B0005464FF1F1722014B1A8070475464FF1F58
:1066C00070B505000E2005F09BF9041E13D0D023F1
:1066D000037000230622837007494570033005F0DC
:1066E00047F8064B2100DA8A62811B7E2373044B34
:1066F000187805F02DFB70BD7064FF1F6064FF1FEC
:106700001443FF1F262803D8024B4000C05A70478D
:106710000148FCE7C642FF1FFFFF000070B50600FE
:106720000C00094D1C220021280005F0A1F9074B9F
:106730001E70074B1C7005F013FB0123002801D0CD
:10674000002312202B7070BD6064FF1F1443FF1FD5
:106750008164FF1F70B505000D4C0800E260A16068
:1067600010220021656005F06BF8012803D110218B
:10677000A06802F058FD10220021280005F060F802
:10678000012803D11021606802F04DFD70BDC046A4
:106790006064FF1F70B5041E05D1002903D00622D6
:1067A0000D4804F0E5FF0D4B1D78012D11D1002C93
:1067B00005D102221A7005F0F3F9280070BD0022FD
:1067C0001A70074B1B78FF2BF7D02000FFF778FFDC
:1067D000F3E70025F1E7C0467064FF1F6064FF1F08
:1067E0001443FF1F030010B5002801D1002010BD85
:1067F00000780B4A002803D15988D1821B7913767F
:106800001378022BF2D10023984200D10333137086
:10681000044B1B78FF2B01D0FFF752FF0120E6E766
:106820006064FF1F1443FF1F002911D000280CD003
:106830004B79012803D140225242134303E03F2207
:106840001340032802D001204B7170474022F4E727
:106850000800FAE770B5094D0100287800280BD030
:10686000074C0622200004F083FF21002878FFF760
:10687000DBFF200005F01CF970BDC0468064FF1FDF
:106880005A64FF1F00290AD0012808D13F224B7902
:106890009343C02B03D0403B5A425341981C70474E
:1068A00070B5174D06002B78FF2B15D00A2005F088
:1068B000A7F8041E10D0D0230370C83B8370114B7F
:1068C00011491B784670C3700622043004F050FF53
:1068D0002100287805F03CFA0C4B1B78012B0DD1D8
:1068E0000B4B1B68002B03D09B68002B00D09847F4
:1068F000084B04211878084A05F092F970BDC0468B
:106900001443FF1F8064FF1F5A64FF1F7C64FF1F36
:10691000A864FF1FAC64FF1F60EA0000014B986889
:106920007047C0466064FF1F014BDB681868704702
:106930006064FF1F074B10B5DA68136801331360FA
:10694000054B1878FF2803D08021C90104F0B0FF5F
:1069500010BDC0466064FF1F1443FF1FF7B50E0053
:1069600002F0C8F8051E1CD00E4B06621F78002FDF
:1069700000D10778AB791020019305F041F8041E8F
:106980000FD0D0230380C73B8370019BE91DC370E8
:106990000622043004F0ECFE21003800E66005F029
:1069A000D7F9F7BD1243FF1F014B18787047C04657
:1069B0008064FF1F054B002805D1054B1A78054B55
:1069C000002A00D1014B18007047C0467064FF1FB9
:1069D0008064FF1F5A64FF1F014B58687047C04610
:1069E0006064FF1F024B1868431E9841C0B2704795
:1069F0008464FF1F421E03000120152A03D9FF3BB8
:106A00005A425341D8B27047F0B51C0000230E0023
:106A100085B0039002920B70029A934201D300203A
:106A200019E0E55C5A1CD2B2002DF8D00298511939
:106A30008142F4DC0233DFB2A35C18000193FFF75C
:106A4000D9FF002807D0013D019A0399EBB23370BA
:106A50008A4202D1E01905B0F0BDDB19DBB2DBE7F9
:106A600010B50C0002F09EF803001220002B03D09A
:106A70002100588804F0FCFE10BD000070B50E4DDA
:106A800084006359002B15D0186A002801D005F046
:106A90002FF82B59586A002801D005F029F82B59F6
:106AA000986A002801D005F023F8285905F020F84D
:106AB00000232B5170BDC0469064FF1F1C4B70B566
:106AC00004000E00150099420AD11A4B1B68002BD6
:106AD00001D1122070BD1B68002BFAD09847F9E74E
:106AE000154B994215D1134B1B68002B0AD01B681C
:106AF000002B07D09847002804D1104B1C70104B76
:106B00001D70E7E729002000FFF7AAFF0028E1D168
:106B1000F3E7080001F0EEFF0028DAD00378032045
:106B2000A342D7D12900300004F0A2FED2E7C0462C
:106B3000FEFF00008C64FF1FFFFF00008964FF1F41
:106B40008864FF1FF7B50400808801F0D3FF00259B
:106B5000A84203D00578A08802F008F81C4E3378CC
:106B6000002B1FD0AB421DD11A4B28001978FFF71C
:106B700077FF002818D000233370A3790820A77866
:106B8000A688019304F03CFF011E0DD0D0230370B2
:106B9000CA3B8370019B477086808371280005F093
:106BA000D7F801E0002DE8D1A0880B4B8200D35824
:106BB000002B01D0FFF762FF1721A088FFF768FDC7
:106BC000A08801F027FDA08801F0FEFDF7BDC046BA
:106BD0008964FF1F8864FF1F9064FF1FF0B587B0B2
:106BE0001D000CAB1B88070001930DAB1B88142004
:106BF00002930EAB1B88160003930FAB1B8800910A
:106C0000049310AB1B88059304F0FAFE041E1AD0FF
:106C1000D0230370CB3B47708370C67006222900D7
:106C20000430002D11D004F0A3FD019B21006381ED
:106C3000029B0098A381039BE381049B2382059B15
:106C4000A37405F085F807B0F0BD04F011FFECE780
:106C5000F7B5009308AB1B8807000C200D00160049
:106C6000019304F0CDFE041E13D0280001F042FF72
:106C700000280FD00078D0232370C93BA370009B5D
:106C800021002381019B6770A580E680638105F068
:106C90005FF8F7BD014B1878EDE7C0461443FF1FBE
:106CA00013B5040064890389C2888188C078009480
:106CB000FFF7CEFF13BD000010B5044C206800287C
:106CC00003D004F015FF0023236010BD9464FF1F60
:106CD000A122F0B5818892004A43384B384F1B6897
:106CE00004009B189D2292009B18827989B01A603B
:106CF0003B68002B5FD01D78324B1B68002B04D003
:106D00005B68002B01D00020984726000836310030
:106D1000E079FFF7B7FD237DE0710200E07804938E
:106D2000638A29000393238A0293E3890193A3884A
:106D300000933300FFF752FFE378002B0BD1E28979
:106D4000A379A18802920196E2792800009201229B
:106D500001F0DAFEE0703B68002B20D0FFF7ACFFBB
:106D6000194D287800281AD0184B1978FFF778FEAB
:106D7000002814D02B78E67808200793A78804F021
:106D80003FFE011E09D0D0230370CA3B46708370BA
:106D900087808671079804F0DBFF00232B70172192
:106DA000A088FFF775FCA08801F034FCA08801F0F2
:106DB0000BFD09B0F0BD064B9DE7C0463409FF1F2F
:106DC0009464FF1FA864FF1F8964FF1F8864FF1F6E
:106DD0001443FF1FF8B5070008000E0001F08AFEFB
:106DE000041E18D02620FFF78DFC051E00D1257843
:106DF000062004F005FE041E0DD00021062204F03A
:106E000037FED0232370C23B21006770A370A68099
:106E1000E8B204F09DFFF8BDF0B585B001930AAB70
:106E20001B78070002930BAB1B7808000D00009243
:106E3000039301F05FFE061E22D0102004F0E0FD57
:106E4000041E1DD01022002104F012FE2620FFF7A0
:106E500059FC002800D13078D0232370C13BA370A7
:106E6000009B21002372019B67706372029BA580C7
:106E7000A372039BC0B2E3720C9BE36004F068FF53
:106E800005B0F0BDF7B50D00019001F033FE071E0F
:106E900020D00E2004F0B4FD041E1BD02620FFF7E6
:106EA00031FC061E00D13E78D0232380C53B06224C
:106EB000A370F91DE01C04F05BFC019B2A006381B8
:106EC0000123DD401A401D40210022736573F0B29A
:106ED00004F03EFFF7BD0000F0B585B00290100051
:106EE0000D0017000A9E039301F004FE041E31D02A
:106EF000029B002B2ED1039B02795B0724D5122322
:106F000013430422002E08D10B99002905D10C99B6
:106F1000002902D10D9900291AD01A430D9B227124
:106F2000002B00D0C9E0002E00D1CFE0002D00D012
:106F3000CCE0606A002801D004F0DAFD1C213000AA
:106F400004F096FE606205E002239A430E33D7E711
:106F500093432371654BBA00D458002C00D1AAE0AA
:106F6000002E10D0236A002B03D11C2004F050FE09
:106F700020625E4BBA00D358186A002803D01C2246
:106F8000310004F0F5FB0C9B002B12D0574CBB00DA
:106F90001D596B6A002B03D1162004F039FE68627C
:106FA000BB00E358586A002803D016220C9904F05D
:106FB000DFFB0D9B002B11D04C4DBC006659B36A12
:106FC000002B03D1142004F023FEB0622B59986AE1
:106FD000002803D014220D9904F0CAFB380001F0F8
:106FE00089FD051E67D0414BBA00D358002B62D0F3
:106FF0001A6A3420002A00D11C389A6A002A01D06B
:10700000143080B20B9A002A01D01C3080B25B6A27
:10701000002B01D0163080B204F0F2FC041E4AD0DE
:107020001822002104F024FD2620FFF76BFB0190BD
:10703000002801D12B780193D0232370029B2000DC
:1070400063700A23294EA370039BBD00A371AB5943
:10705000A780196A1830002905D01C22A06004F00E
:1070600087FB200034307359996A002907D0030048
:1070700014221433E060029304F07AFB02980B9B15
:10708000002B08D003001C221C330B9920610293B3
:1070900004F06EFB02987359596A002903D0162236
:1070A000606104F065FB6B462100187904F050FE26
:1070B0003800FFF7E3FC05B0F0BD10220D9B0D99E1
:1070C0001B69A018236204F053FB2CE70B9B002BD9
:1070D00000D13FE7012D00D03CE7606A002801D0D5
:1070E00004F006FD1C210B982AE7C0469064FF1FA0
:1070F00010B5044C2068002803D004F0F9FC0023EC
:10710000236010BD8464FF1F0B4B07B51A68002A6B
:1071100001D100200EBD6946531C012012780731B1
:10712000FFF772FC0028F4D0027801231000184009
:107130001A42EED0EEE7C046A064FF1FF0B51F4F25
:1071400001203B6887B0002B25D09B78059300F089
:10715000B3FB002821D00A20FFF7D4FA04000B204B
:10716000FFF7D0FA164B05001E78731E9E413B6850
:10717000F6B2191DD878FFF757FB3B682900DA7A79
:10718000043303929A790193029200903300200015
:10719000059A04F03DFB07B0F0BDFFF7B5FF0028EE
:1071A00005D00620FFF7AEFA04000720D8E7082034
:1071B000FFF7A8FA04000920D2E7C0468464FF1F45
:1071C0008064FF1F70B50A4E040033780D00FF2B5A
:1071D0000DD0042004F014FC011E08D0D02303704D
:1071E000CE3B45708370C470307804F0B1FD70BD43
:1071F0002443FF1F70B5040006200D0004F000FCBE
:10720000011E0AD0D0230370CD3B8370054B447020
:107210001B688580187804F09BFD002C01D0FFF7D7
:1072200067FF70BD8464FF1FF8B5264F06003B68FA
:107230000D001124002B05D10522234B1B7813428E
:1072400002D112242000F8BD204A10241268002A1E
:10725000F8D01278002AF5D0DB0719D52B789A1EC2
:10726000012A1AD80C2004F0D3FC1324386000281B
:10727000E8D000230A22437029000670023004F08F
:1072800077FAFFF75BFF041E0AD0FFF731FFD9E75B
:1072900000F012FB0028E1D1E4E7002BE2D0D0E7B8
:1072A0000B4B1B78032BCDD11D20FFF72BFA094B7D
:1072B00018800028C6D0084B04211878074A04F02B
:1072C000AFFCBFE78464FF1F8164FF1FA064FF1F42
:1072D0008064FF1F7E64FF1FAC64FF1F60EA000034
:1072E000F7B50193194B14001A78052306000F0017
:1072F00012201A4221D0012920D1154B1D68002DE2
:107300001BD002201F2C18D8002C02D0019B002B70
:1073100013D0104B1F221E706E1C0021300004F091
:10732000A7FB01992200300004F022FA310020006E
:107330002C70002F06D004F003FBFEBD064B12207C
:107340001D68DCE704F034FDF7E7C0468164FF1FE9
:10735000A064FF1F2443FF1F9C64FF1FF8B50F4E5E
:1073600012243368002B17D01B780F3C834213D1B3
:1073700000250B4F0221387804F092FC094B0421C0
:1073800038781D8004F08CFC074B28001D80336882
:107390005C7004F045FB04002000F8BD8464FF1F0E
:1073A000AC64FF1F9864FF1F7E64FF1F70B5012847
:1073B00023D11B4C2388002B03D01A4A1578002DAB
:1073C00007D0194B1B68002B02D01878FFF7C6FFB7
:1073D00070BD3B2B02D93C3B2380F9E7134E0221C1
:1073E000307804F05DFCFA222388920002215A438F
:1073F000307804F0E5FB2580EAE70B4B1B68002B97
:10740000E6D00B4B1B785B07E2D5084B02211878BE
:1074100004F046FC0022024B1A80FFF769FED7E712
:107420009864FF1F7C64FF1F8464FF1FAC64FF1F10
:107430008164FF1FF8B51E4D2868002803D004F0B2
:1074400057FB00232B601B4E3068002803D004F04C
:107450004FFB00233360184F05243B781800204071
:10746000234221D0154800F02BFA3B78234213D059
:10747000202004F0CDFB2860002813D0202200211A
:1074800004F0F6FA202004F0C3FB041E306005D09F
:107490002022002104F0ECFA002004E0286804F027
:1074A00027FB2C601320F8BD00F00AFAF4E7C04671
:1074B000A064FF1F9C64FF1F8164FF1F1843FF1F10
:1074C00010B50A4C23681A1E0ED0002808D10130CE
:1074D000587004F0A5FA002805D02368002B02D0CC
:1074E0000021FFF787FE0122100010BD8464FF1FFA
:1074F000F7B5274E050033680191181E21D05C783E
:10750000244F012C30D1FFF7FFFD002825D02000AB
:10751000FFF7F8F80400412814D91F4B022118780E
:107520001E4A04F07DFB1E4B3C3C1C80022233684B
:107530005A703B78002B14D128000199FFF75AFEAE
:107540000120FEBDFA2292004243002AEED0124BE7
:107550000221187804F034FBE8E7FFF7D3F80200C3
:10756000F3E700233B70EBE73B78002BE8D10320E7
:1075700004F046FA011E08D0D0230370CC3B4570BE
:1075800083703368187804F0E3FBFFF7B1FDD7E7A9
:107590008464FF1F7C64FF1FAC64FF1F60EA00006F
:1075A0009864FF1F10B51749838802008B4220D0D2
:1075B00011D815498B4217D0144900205B1899B295
:1075C000012907D8926811785A425341D8B2FFF77F
:1075D000F9FD012010BD0E4A00209B1807229BB226
:1075E0009A424041C0B2F5E783681878FFF768FF18
:1075F000F0E7836899785A78090218781143FFF701
:1076000077FFE7E70A20000006200000F8DFFFFF11
:10761000AFDFFFFF014B18707047C0462543FF1FC7
:1076200010B5064C207001F041FA207804F070FA91
:107630000521207800F062FD10BDC046AC64FF1F3C
:107640000BB273B50D00002B00DBC4E0884B18783B
:1076500004F0BEF9041E0ED00378912B0FD0A22B9C
:1076600000D1A1E0834B1878FF2852D0210004F00C
:107670006FFB00284DD180200002684076BD437822
:107680000F2B76D013D8052B70D00E2BEAD1808823
:10769000794B98422BD8794B98421BD8784B98421B
:1076A000E0D1A3681878591CFFF774F838E03E2B36
:1076B000D8D18378032B74D06CD8012B6ED0022BD9
:1076C000D0D1704B1B68002B23D05B68002B20D0DF
:1076D00098471EE06C4BC0180C28C3D804F0E0F9A2
:1076E0001DC2C2150BC20B0B0B3223C23C00674BF1
:1076F000C0180728B6D8664B1B68002B09D01B683A
:10770000002B06D0200098470AE0A3681878FFF7FE
:10771000C7F8200004F024FAADE7A068FFF762F88C
:1077200000289FD0F5E7A3681B78002BF1D0554BBC
:107730001B68002BEDD01B68002BEAD021005548B8
:107740009847EDE74F4B1B68002BE2D01B68002BDE
:10775000DFD021005048F3E7504B1B68002BD8D0F6
:107760005B68002BD5D021004348E9E7FFF7EAF931
:10777000CFE780884A4B984203D04A4B984200D0CA
:1077800070E7464B1B68002BC3D05B68002BC0D052
:107790002100D5E7153B012BBBD963E7FFF798FA2A
:1077A000B7E7FFF77DFAB4E73F4B1B78042B07D10F
:1077B00000236A4613800179408800F0C5FCA8E7E1
:1077C000364B1B68002BA4D05B68002BA1D00100B6
:1077D000364898479DE7012421420AD0294B1B686F
:1077E000002B04D05B68002B01D0002098470120BB
:1077F00043E78B070AD5264B1B68002B04D05B6838
:10780000002B01D020009847022036E704212800F1
:1078100008400D4200D131E7254E3388002B21D09E
:10782000013B9BB23380002B1AD1FFF7DBF8002815
:107830000AD0204B1C70164B1B68002B04D05B68D1
:10784000002B01D020009847FFF7C6F8694601F0E9
:1078500001FD6846FEF7FEFF1D20FEF753FF308056
:1078600004200AE7024B187804F01AFAF8E7C04639
:10787000AC64FF1F2543FF1F0E2000000120000005
:1078800009100000A464FF1FFEDFFFFFAFDFFFFF52
:10789000A864FF1F0C2000000B2000008C64FF1F59
:1078A0000D200000132000008164FF1FFFFF000077
:1078B0007E64FF1F7C64FF1F10B501F09BF910BDB3
:1078C000014B18607047C046A864FF1F0B8800205A
:1078D000162B01D817230420014A13807047C04695
:1078E0005664FF1F00207047074A03001188814239
:1078F00007D091880020994202D1013080001018F1
:1079000070470020FAE7C046B464FF1FF0B58F78D7
:1079100006000D00C5B01E2F15D1FFF7E5FF051EAF
:1079200003D10024200045B0F0BD00223B0031000F
:10793000C078009200F0B2FB0400A81C00F0D2FB5B
:10794000FF23EB70EEE7264B062403931B78FF2BF7
:10795000E8D0182FE6D87B08224A013BDB000292D0
:107960009A589446002ADDD0029AD3185B68002BFF
:10797000D8D00878002802D14B78012B02D10624F8
:10798000122FCFD107AFAB88697800976446AA68F9
:10799000A047041EC6D1AB78029A5B08013BDB000E
:1079A000D318390030005B689847041E0BD1AB78C0
:1079B000042BB6D0039A310010782200009700F013
:1079C0006DFB0400AEE76A78002AABD1AA7805A95E
:1079D0003B88087130000A704B80FEF747FBA0E738
:1079E0002843FF1FB8BF00111D4B37B50500984253
:1079F0000BD000290AD1FFF777FF002805D11948DD
:107A0000FFF772FF002800D0058037BD01291AD189
:107A1000FFF76AFF041EF8D001235B420380A378BE
:107A2000FF2BF2D0FE2B07D00023E0781422009326
:107A300029001E3300F032FBA01C00F053FB012391
:107A40005B426380E1E70229DFD1013901F0BEF832
:107A50000028DAD12800FFF747FF041EDFD1D4E762
:107A6000FEFF0000FFFF0000022210B5074B52424C
:107A70001A80074801325A809A80DA8000F07EFA34
:107A8000044801F025F8002010BDC046B464FF1F73
:107A90000D790011E97900110388F7B50400002B76
:107AA00002D102252800FEBD426802211378254834
:107AB0005268FEF7A5FD00282ED0234F01253A88F5
:107AC000002AEFD0802321885B0201259B1A99426E
:107AD000E8DC0C2004F09CF8061E31D03B8822889C
:107AE0009C4600231800019561469DB2491989B250
:107AF000AA421BD8002801D062443A8000233000FB
:107B0000082208C0210003F033FE104A1368002B3E
:107B100013D100251660C5E76268022113780C486E
:107B20005268FEF76DFD0028C7D1BAE760681D01F5
:107B30004019418101330198D6E71A001B68E6E736
:107B40001325AFE726C000112643FF1FB064FF1FB7
:107B500024C00011014B18707047C0462843FF1F16
:107B600014230A0010B51A40194204D00122102132
:107B700001F048F810BD4B06F9D4012088434000BD
:107B8000F8E710B514008B0604D50122102101F08E
:107B900039F810BD08230A001A40194202D14BB22D
:107BA000002B0FDA102101F02DF8002808D0230057
:107BB000F2331B78002BECD0F1342378012BE8D181
:107BC0000020E6E703208907FAD4E2E7F0B51F00BA
:107BD000184B85B01C68019002910392002C27D1AC
:107BE000200005B0F0BDA5683301ED186B89019A3E
:107BF000934211D3029A93420ED8002F04D10A9BCC
:107C0000002B10D12C00EBE73B002978039A686821
:107C1000FEF7F6FC0028F2D10136B6B2A388B342D3
:107C2000E1D82468DAE7A3680A9A5B891380E9E758
:107C30000026F3E7B064FF1F37B50C000A884988B7
:107C40000123914217D3002A15D0651D23792A00FC
:107C500002210A48FEF7D4FC102300280BD0237918
:107C60006188208800242A000094FFF7AFFF0A23D0
:107C7000A04200D0230018003EBDC04626C000111F
:107C800013B50A0008884988012388420BD80028C8
:107C900009D00024137905320094FFF797FF0A23D7
:107CA000A04200D02300180016BD13B50A000888B2
:107CB0004988012388420BD8002809D00024137971
:107CC00005320094FFF782FF0A23A04200D0230070
:107CD000180016BDF0B58BB003904A8808880E00D6
:107CE0000123824255D3002853D00023012704AC3E
:107CF00023700022718813000092FFF767FF051EB2
:107D00003ED02078002835D12B78022B18D167700F
:107D10006A8983000130E31880005A806968022272
:107D2000201803F025FD23780133DBB22370042BE8
:107D300019D93B006889013080B2002BD9D01FE0EF
:107D400002236370122358436A89231804305A802F
:107D500069681022201803F00BFD23780133DBB291
:107D60002370002BE5D10C4A6B899B185A42534172
:107D7000DBB2DFE76378012BE4D12B78022BC7D08D
:107D800022780A23002A04D021000398FEF798F9EC
:107D9000002318000BB0F0BD0100FFFF0F4BF0B542
:107DA00004001868002816D083685D89A54207D8AA
:107DB0008288AE18B44203DA12019A18934201D1B4
:107DC0000068EFE71E005F891036A74204D1002942
:107DD00000D00D801800F0BD3300EFE7B064FF1F46
:107DE00070B505000C0008880021FFF7D7FF0300DD
:107DF0000120002B04D022002800197AFFF7C1FED1
:107E000070BDF7B50C00002501902300EE331B7800
:107E1000AB4201D800200AE06B00E65A0021300096
:107E2000E718FFF7BBFF002802D126800130FEBD16
:107E3000017A0198FFF794FE002802D03B88238046
:107E4000F5E70135EDB2E0E710B504000888002140
:107E5000FFF7A4FF03000120002B03D02000197AB4
:107E6000FFF77EFE10BD0000054B1B68002B01D103
:107E7000180004E09A6852898242F6D198887047C7
:107E8000B064FF1FF0B50E27002687B0039302AB46
:107E9000FF183E8005001F4B40891400984207D010
:107EA0002B78013000976A6880B2FFF78FFE0600DA
:107EB00002212B7818486A68FEF7A2FB00280FD031
:107EC0006C892000FFF7D0FF002802D0013C041984
:107ED000A4B2039B002B00D01C80300007B0F0BD83
:107EE00002212B780D486A68FEF78AFB0028E7D14B
:107EF00002212B780A486A68FEF782FB002807D027
:107F0000002EDED03B88A342DBD17489013CDFE741
:107F10006C89DEE7FFFF000026C0001124C00011BD
:107F200022C0001110B50C00FFF7DEFC0300022098
:107F3000002B0AD0002C00D023609B781720FE2B4A
:107F400003D00138FF2B00D1002010BD73B50D0008
:107F500001A904001600FFF7E5FF172805D0002E41
:107F600004D129002000FEF727F976BD0122102157
:107F7000200000F047FE0028F3D0F6E7014B186020
:107F80007047C046C064FF1F37B56B469D1D01009A
:107F900004000222280003F0C3FE2B88B02B0ED170
:107FA0002379122B09D12300FA331B78012B06D138
:107FB0000121608800F0E0F801E01B2BF8D037BD0C
:107FC00010B5054B0421187000F098F8FFF74CFD30
:107FD000FEF770FB10BDC046C464FF1F0020F0B563
:107FE0000BB20F0087B0834234DA274B187803F0C6
:107FF000EFFC051E2BD00378A02B25D103AE31005A
:10800000FEF7E4F8041E0BD1B378DB0724D51F4B31
:1080100006341B68002B03D03100688898470400A1
:10802000A868002801D003F0E3FD002C08D1184A0D
:10803000039B1340174A934206D0B3781B2B03D0FF
:108040000121688800F098F8280003F089FD80205D
:108050000002784007B0F0BD0F4B1B68002B10D01A
:10806000310068889847041EDAD07378002BD7D186
:10807000B27801A90A704B800C716888FDF7F6FF91
:10808000CEE70624F1E7C046C464FF1FBC64FF1FAF
:1080900000FFFF0000011200C064FF1FF7B5019050
:1080A000FC200D0017001E0003F0AAFC04001320A2
:1080B000002C12D0B02320002370089BF42267709C
:1080C000658026710830002B08D0190003F050FBA2
:1080D0002100019803F03CFE0020FEBD089903F04A
:1080E000C7FCF5E710B5041E06D00078FD2803D8BC
:1080F00003F0A6FCFF23237010BD00000A1F93B2FB
:1081000010B504000220032B05D882400020024B4A
:10811000D1529B189C7010BDE464FF1F0B8870B592
:10812000043B04000D000220032B0BD8012120008A
:1081300000F04CFD03001420002B03D02900200088
:1081400000F0DEFB70BD000007B51300034A00928B
:108150000A00012100F02CFC0EBDC04685830011F1
:1081600007B5019203220092024B0A00122100F08F
:1081700049FC0EBD0384001107B56B4601AA1180AE
:108180000449D88008780633012802D1190003F089
:10819000F7FB07BDC564FF1F0C4B10B5187000231B
:1081A000FF210B4A1380138193819380094A5380E6
:1081B0001370517293819372D174D3821375517776
:1081C00003F08EFC00F0FCF910BDC046F464FF1F04
:1081D000E464FF1FC664FF1FF0B58DB06B4600203E
:1081E00003910C229B5E834200DBB0E05D4B18786C
:1081F00003F0EEFB051E00D1A4E00378902B00D025
:108200009DE006AF01004688380000F013FA796857
:108210000400002900D19CE03B88052B6ED13B89EE
:10822000032B1CD905AC200000F0A2F86288172AA5
:1082300061D83989131D994231D179682378043185
:108240000291D90738D5607800F08EF9071E06D064
:10825000002303712378012B08D0132B23D0A868A7
:10826000002800D178E003F0C3FC75E06288029931
:1082700009A800F0A6F80290380000F08BF909AACE
:108280002378387A0192002231000092029A00F09D
:1082900012F9380000F064F9029B002BDFD03000A7
:1082A00000F080F9DBE70378032BD8D162880299CC
:1082B00009A800F0D6F8DEE7122B13D1029909A81D
:1082C00000F0B5F8021EEAD127498B88002BC6D0F2
:1082D000887909A92378019161780091310000F033
:1082E000EAF8BCE7002302AA93833000617809AA68
:1082F000FFF72AFFB3E71D4B0993F6E7042B02D0E3
:108300009A1F012AABD8184A043B9B00995A0029AE
:10831000A5D0D218907831003A0000F0AEF80028CD
:108320009DD13B88042B03D001213000FFF724FFAF
:10833000012C04D1A868002801D003F059FC2800C2
:1083400003F00EFC8020039B0002434018000DB098
:10835000F0BD012800D182E701213000FFF70CFFBA
:10836000EDE7C046F464FF1FE464FF1F010017003F
:108370000B7803704B784370CB788A781B021343D9
:10838000438070470A88030002700A88120A42700C
:108390000A88012A06D14A8882704A88120AC27065
:1083A0000420704702208242FBD14A8804309A7030
:1083B0004A88120ADA708A881A718A88120A5A71EF
:1083C000EFE710B50400012082420CD94B780A78FF
:1083D0001B0213432380834206D1CB788A781B0289
:1083E00013436380002010BD022BFBD1CB788A7829
:1083F0001B02134363804B790A791B021343A3804A
:10840000F0E70B8803700B881B0A43704B8883705E
:108410004B881B0AC3708B8803718B881B0A4371BE
:10842000CB888371CB881B0AC37108207047030077
:108430000120082A14D14A780878120202431A80CF
:10844000CA788878120202435A804A79087912025F
:1084500002439A80CA798879120202430020DA80A6
:10846000704710B504000120022A05D100204B7886
:108470000A781B021343238010BDF8B506001020B4
:108480000F00150003F0BCFA04000120002C0ED0F0
:10849000A0230C22290023806780201D002D07D0F7
:1084A00003F066F92100300003F052FC0020F8BD13
:1084B00003F0DEFAF6E7F7B51E00009008AB1420D3
:1084C00017001D78019103F09BFA041E12D0A2231D
:1084D0000370019B47704380099B057146710C2214
:1084E0000830002B07D0190003F042F92100009852
:1084F00003F02EFCF7BD099903F0BAFAF6E737B599
:10850000041E0FD04388002B0CD00025C1881323F4
:10851000007A172201950095FFF7CDFFFF236580B4
:108520006372257037BD000010B50C4904004A88FD
:10853000002A09D08B89002B05D00020CB8A02228B
:10854000834201D010BD012213000A2043430020C2
:108550004032C854C81842800472F3E7C664FF1F53
:108560000023438003707047094B00211A0010B5A7
:108570005C88002C06D01C79844203D10A234B432B
:10858000D01810BD01310A330329F1D10020F8E7DA
:10859000C664FF1F10B50400407A03F051FAFF23B0
:1085A000637210BD7047043010B580B203F070FAEA
:1085B000002803D00421494203F002F910BD000055
:1085C00070B50025104CA0682580A581A580A84223
:1085D00002D003F00DFBA56000250C4C0C4B606D28
:1085E0001D80230058331D70A84202D003F000FB09
:1085F000656500256068002801D003F0F9FA0135AF
:1086000008340A2DF6D170BD8C65FF1F3065FF1F41
:108610008065FF1F70B5041E09D1054D2880A88113
:10862000A880A868002802D003F0E2FAAC6070BD10
:108630008C65FF1FF0B54B8885B001930023436024
:108640000A7905000F00022A00D07BE0CA88032ABD
:1086500017D98B685E7819783602DC78D8790E43A2
:1086600099781B7A24021B020C43034353495BBADB
:108670000B80331D93421ED1042C04D0631F022BA8
:108680000ED9012015E0019A4D4B1201D35A002B4F
:1086900006D00198FFF7BEFF4A4A13690133136100
:1086A0000421B8682E812C80494203F089F8686063
:1086B000002005B0F0BD434D042C06D0631F022BF3
:1086C0000FD9EB680133EB60DBE7019A3C4B1201F9
:1086D000D35A002B05D00198FFF79CFF2B6901337B
:1086E0002B61374B30000293019B029A1B010193CF
:1086F000002301998C468B52130063449C800393A2
:108700009E81FFF750FF039B041E986016D0042142
:10871000B868494203F054F8FA880100043A20008E
:1087200003F026F80199029AFB888A5A043B9B18A9
:10873000029A8B522B6801332B60A2E7AB6901339D
:10874000AB619EE71E4B0293019B1E01029BF35AF5
:10875000002B2DD002998C19A068002828D0012A5E
:1087600026D1FA889B189BB27352A189994217D3DC
:108770009B1AC018B96802F0FBFF029BA289F35A4A
:10878000934200D07DE700222B81A3882B80A36831
:108790006B60029BF2520B4A53680133536070E7DF
:1087A000084A9368013393600198FFF733FF68E745
:1087B000044A536901335361F6E7C046F664FF1F6C
:1087C0008C65FF1FFC64FF1F70B5051E15D10B4C97
:1087D0000B4B1880230058331870606D002802D0AE
:1087E00003F006FA6565250050356068002801D061
:1087F00003F0FEF90834AC42F7D170BD3065FF1FBD
:108800008065FF1FF0B51700A12285B0920001938B
:108810004243394B06001B680C009B18D933FF33C9
:108820001D78FDF741FF0430854204DD3000FDF77F
:108830003BFF0430C5B2BD4207D33A0000213000EF
:10884000019B02F0A5FF05B0F0BD2900380003F040
:1088500017FA2300C6B250331E700393019B290000
:108860006365380003F03CFACBB20293002B02D0D0
:10887000039B01361E7000262300503303931B78A0
:10888000B34204D8606D002831D10020DBE7029AA2
:108890002800002A04D0013B1000B34200D0280079
:1088A000F700E719387003F0ABF9786000280ED0B4
:1088B0003A78019902F05CFF019A3B780136D318AF
:1088C0000E4A0193D369F6B20133D361D4E7039B17
:1088D00018706065A74205D1084A1320D36A013396
:1088E000D362B0E7606803F083F90834F2E703F07D
:1088F0007FF900236365C8E73409FF1FFC64FF1F8D
:10890000F7B50D0007000421686802F059FF2B89B4
:10891000040003702B891B0A43702B8883702B88FB
:108920001B0AC3702E8902250436F6B2F42E15D820
:108930001B4B9F4214D10C2003F062F81135011E2D
:108940000CD0902303708E3B0371043B4380154B86
:108950008460C680187803F0FBF900252800FEBD6E
:108960005C237B43104AD3180093583301931B7840
:10897000002B0FD10300320038000099FFF742FFAF
:10898000019B05001B78002BE8D13800009902F00C
:108990005FFFE3E7054A0725536A01335362DDE7CA
:1089A000FEFF0000F464FF1F3065FF1FFC64FF1F23
:1089B000F0B587B0009017200F0016000193FFF765
:1089C000F2FD1325041E19D00C98031E02D0019944
:1089D000201D9847030AE370052302AAA070043003
:1089E000908127700098667003A993800494FFF724
:1089F00087FF051E02D0200003F0FAF8280007B018
:108A0000F0BD0000F0B587B01F000CAB1B780391E0
:108A1000059301210DAB06001C78049200F0D6F8F6
:108A20001425002821D02000FFF77EFD0135041E0B
:108A30001BD01149059B0A7803700132D2B2131E74
:108A4000C68001D101231A000B7022713000049BF3
:108A500003990097FFF7ACFF051E09D12300210001
:108A60000648074A093303F033F9280007B0F0BD80
:108A7000002363802370F8E7F864FF1FFF84001170
:108A800030750000F8B505000E00064C064F23684F
:108A9000002B02D03100280098470434BC42F6D1A4
:108AA000F8BDC0469C65FF1FB065FF1F0123064A45
:108AB0005B425380002313715362044A1360536076
:108AC0009360D36013617047B065FF1F9C65FF1F03
:108AD0000200002310B506499C000859002801D166
:108AE000625010BD0133052BF6D11320F9E7C046C3
:108AF0009C65FF1F034A5388181A4342584140425D
:108B000010407047B065FF1FF0B585B002930AAB07
:108B10001F780CAB1B88009008000E000192039395
:108B2000FFF7E8FF05001120002D1BD10E48FFF7CD
:108B3000E1FF04001520002C14D006220B99A77128
:108B4000E01D02F015FE019B30002371029B2900FD
:108B50006371009B66802370039B6562E381FFF76E
:108B600091FF280005B0F0BDFFFF000010B5FFF732
:108B7000C1FF04000220002C12D060880121FFF701
:108B800081FF606A002801D002F0B2FF2822002194
:108B9000200002F06DFF012300205B426380207102
:108BA00010BD000030B5074A074C55880100137806
:108BB0000020A54204D05B1A59424B415842104054
:108BC00030BDC046B065FF1FFFFF0000084A10B56A
:108BD00001230C00904208D0FFF78CFF031E04D045
:108BE000037923405A1E9341DBB2180010BDC046E2
:108BF000FEFF0000024B1879431E9841C0B2704737
:108C0000B065FF1F70B504000D001600FFF772FF7E
:108C1000002804D10D4B9C4200D0143070BD416A35
:108C200003790520002907D012221A40102A02D108
:108C30000520002EF2D10F20DB06EFD5897E0C2017
:108C4000A9428941494249420840E7E7FEFF000046
:108C5000030010B5002800D110BD0348034A418825
:108C60009142F9D09847F7E7B065FF1FFFFF00007A
:108C7000002330B5C45CCD5C6C40D4540133102B60
:108C8000F8D130BD0F23002210B5C45C640022432C
:108C9000CA54C25CD209013BF7D210BD02000100E8
:108CA00010B52032103102F0F3FD10BDF0B58BB0DD
:108CB0000390102005931700049102F0A9FF009083
:108CC000102002F0A5FF009B13240190002B05D07B
:108CD00000280CD11324009802F00AFF019B002BFE
:108CE00002D0180002F004FF20000BB0F0BD1020ED
:108CF00002F08EFF0600102002F08AFF1324050008
:108D0000002E00D1AEE0002819D01022002102F080
:108D1000AFFE32002900039802F0BAFD041E0ED106
:108D200033787F2B51D830000099FFF7ABFF009BC1
:108D30001B787F2B53D801990098FFF7A3FF3000D1
:108D400002F0D6FE002D02D0280002F0D1FE002C49
:108D5000C1D1102002F05CFF0600102002F058FF85
:108D60000290002E7CD0002878D03A000F322300E9
:108D70000125121105D00F333B4015B25A42534121
:108D80001BB26A1E1201002B33D0049BD2B298187A
:108D90000099029AFFF76CFF013D1022002130007C
:108DA00002F066FEADB2049F2D017D19AF4242D0A4
:108DB000002C33D0300002F09BFE029B002B00D130
:108DC00089E7180002F094FE85E729003000FFF7DC
:108DD00059FF28002549009AFFF74AFFA7E7290015
:108DE0000098FFF74FFF28002049019AFFF740FF46
:108DF000A5E70F210F4004998A18D9B28F4208D9EC
:108E0000D15C06A819540133102BF6D1029A0199AE
:108E1000C0E7791A48424141C901F2E73900300000
:108E200006AAFFF725FF3200039806A902F030FDDD
:108E300010370400BAE7002CBCD13000029906AA12
:108E4000FFF716FF320006A9039802F021FD082261
:108E500004003100059802F08BFCABE71324A9E76E
:108E60001324AAE7002800D06EE733E72CC00011D6
:108E7000F0B58BB00F0016000225009000283FD0FF
:108E8000002A3DD00B1DDBB21800029302F0C0FE99
:108E90001135041E34D0FDF747FD05003A00009956
:108EA000201D02F09DFEEBB20393E3702B0CDBB2AE
:108EB0002F0A00936370FFB22B0E2370A7700193EB
:108EC000FDF72CFD1022010006A802F089FE21000A
:108ED000029A04AB06A8FFF7E9FE051E0DD1039B1D
:108EE00008223370009B04A9B370019B7770F37064
:108EF000301D02F075FEFDF71DFD200002F0F8FDAB
:108F000028000BB0F0BDF0B58FB00D00149E03909B
:108F100004920593002A03D1022420000FB0F0BD73
:108F2000002EF9D00398FFF7E5FD1424071EF4D0B6
:108F30007278337812021A43B3781B041343F27821
:108F400012061A43036A0192934201D30133E3D11B
:108F5000002D03D03B7901249B07DED50822002198
:108F600006A802F085FD059B13240433DBB218002C
:108F7000029302F04DFE051ECFD0059A04990430ED
:108F800002F02EFE04223100280002F029FE3900F2
:108F9000102210310AA802F023FE2900029A06AB23
:108FA0000AA8FFF783FE041E0FD1082206A908A80D
:108FB00002F016FE0822311D08A802F061FC01280B
:108FC00007D101990398FDF7C9FC280002F090FD34
:108FD000A3E70124F9E7000070B51C4C05002368E5
:108FE000181E10D0002D14D11A78002A0CD1981C0C
:108FF000083202F0BDFB02F083FC0135002808D1E5
:1090000023681D70012070BD0A331800082202F089
:10901000AFFB2368002BF5D0122002F0F1FC061EF6
:109020000DD0C12321680370457002311022023037
:1090300002F09EFB23683100587802F089FE206818
:1090400002F056FD00232360DCE7C046D865FF1F11
:10905000F8B504002020FDF755FB0D4EA700BB59C5
:109060000500002B0DD000280BD0D878FF2809D19F
:1090700008492A000C55F35907480333611802F0D8
:1090800027FEF8BD290002F08BFC0028F0D1F8E79C
:10909000F465FF1FDC65FF1FA9A2001170B5064D26
:1090A00084006359002B05D0D87802F0C9FCFF2258
:1090B0006359DA7070BDC046F465FF1F70B50600D5
:1090C0008CB00C00150000213022684602F0D0FC64
:1090D00031001022684602F083FD1D20210003228A
:1090E000684402F07DFD6846FFF7D8FD2D2104009D
:1090F00003222800694402F073FD20000CB070BD0B
:10910000F0B50700160097B001931CAB1D78302214
:109110001EAB00910AA800211C7802F0A9FC1022C5
:1091200039000AA802F05CFD1022002102A802F01A
:109130009FFC0722310002A802F052FD072202AB79
:109140009818631E9C41019902F04AFD02AB9C7382
:109150002B005A1E934102AAD3730021102206A8A5
:1091600002F086FC06221D9907A802F039FD1A209C
:1091700002ABC01806221F9902F032FD102200999E
:109180000EA802F02DFD102202AB0EA908781C7863
:10919000013A6040D2B2087001330131002AF5D1A2
:1091A0000AA8FFF77BFD102212A904000EA802F006
:1091B000DFFA102206AB0EA908781D78013A684044
:1091C000D2B2087001330131002AF5D10AA8FFF7A5
:1091D00065FD044310222098E4B212A902F000FDBC
:1091E000200017B0F0BD70B50E0014008CB0010067
:1091F000102268461D0002F0F3FC3100082204A88A
:1092000002F0EEFC2100082206A802F0E9FC684604
:10921000FFF744FD04001022280008A902F0E0FC3A
:1092200020000CB070BDF8B506000D000024371901
:10923000AC4200D3F8BD02F043FB030A3B70631C51
:10924000DBB201379D4203D90234F054E4B2EEE7B9
:109250001C00EDE773B506000C000225002819D0AC
:10926000002917D0032101A8FFF7DDFF6B469A798B
:109270003F231A40013313436A463000937101A91A
:109280002200FFF71BFF051E04D10322E01C01A9E9
:1092900002F06EFA280076BD03785807DA08C00F8E
:1092A000D20080009B0710439B0F1843C0B2704749
:1092B00007230B40C908C9000B4303707047000027
:1092C00070B50400FFF7EAFE134DA4006359002BAC
:1092D00021D0186A002801D002F00AFC2B59986EA0
:1092E000002801D002F004FC2B59D86E002801D0D0
:1092F00002F0FEFB2B59186F002801D002F0F8FB9A
:109300002B59586F002801D002F0F2FB285902F0C7
:10931000EFFB00232B5170BDF465FF1F0E4B800047
:10932000C35870B50C00002B0FD09D68002D0CD0D9
:109330002B78201D0B706B784B70A97CFFF7B8FF62
:109340002B7E23726B69E36070BD10220021200028
:1093500002F08EFBF8E7C046F465FF1F014B186072
:109360007047C046F065FF1F074A0300800082581F
:1093700010B5002A06D0D088984203D1012901D126
:10938000FFF79EFF10BDC046F465FF1FF0B5264EE7
:1093900095B087000B93BB590500099112200A92E2
:1093A000002B31D0D888FFF7A5FB04001420002C37
:1093B0002AD0280010A9FFF7B1FFBB591E781D6AFB
:1093C000002E23D00895FDF7EFFA07000020FDF7E7
:1093D000F1FA0790A379E61D069310AD0CA9089841
:1093E00000F0E2FA0EA9280000F0D7FA0B9B0A99C8
:1093F0000493069B09980293079B03960193009799
:109400000EAB0CAAFFF77CFE15B0F0BDFDF7CCFA51
:1094100006903000FDF7CEFAE31DA779079310AB55
:1094200006000893DAE7C046F465FF1F30B50C4C20
:1094300085002A59030085B00120002A0ED01800AB
:109440006946FFF76BFF2B591A78D888054B002A1D
:1094500000D1054B6A46072100F0D9FB05B030BDAD
:10946000F465FF1F9B990011A999001130B5094CB3
:109470008500295985B010226846253102F078F917
:109480002A591121044BD0886A4600F0C0FB05B070
:1094900030BDC046F465FF1F459A001130B5094C38
:1094A0008500295985B010226846353102F060F9EF
:1094B0002A591121044BD0886A4600F0A8FB05B058
:1094C00030BDC046F465FF1F839A0011F7B54D4FBC
:1094D00086001020F4590D0002F09AFBF359206227
:1094E000186A132200286CD0033A29009C6802F005
:1094F0003FF9F3591A780192002A58D11E6A227D49
:10950000317B944651400122019F114201D16746AF
:109510001740217D914339432175377B4F40BC462D
:1095200060460027800701D44F0817400121022020
:109530008F40227D82433A432275377B5740BC4699
:1095400060460027400701D497080F400420227D81
:10955000BF0082433A432275627D002794466046ED
:10956000727B42400A4201D167460F400121627D71
:109570008A433A436275777B5740BC466046002772
:10958000800701D457080F400220627D7F0082438C
:1095900017436775767B00227E40760701D4BA08B0
:1095A0000A400426617D9200B1430A4362756A78DD
:1095B000002A08D06278002A05D005220533DA7720
:1095C00000221000FEBD04222979114205D1A17CA0
:1095D000114202D10533033AF1E7019A21782C7840
:1095E000002A02D10A002100140018220429E8D818
:1095F000042CE6D805206043034A05331218525C58
:10960000DDE7C046F465FF1F3CC0001110B50A003D
:109610001121024B00F0FBFA10BDC046DF9A001189
:109620000B0030B587B001AD2B806B4604001100F4
:10963000981D082202F09CF82A000B212000024B02
:1096400000F0E5FA07B030BD079B001110B50A0025
:109650001121024B00F0DBFA10BDC0465B9B0011EC
:1096600013B50B0011006A4613706B460400062206
:10967000581C02F07DF86A4608212000014B00F0DA
:10968000C6FA13BD7B9B001110B50A001121024BD5
:1096900000F0BDFA10BDC046CB9B00117FB50500A0
:1096A0000B4BAA00D4580800002C0FD0666F237F04
:1096B000E28821780396266F0296E66E0196A46EE4
:1096C0000094FDF709FC2800FFF7FAFD7FBDC046B6
:1096D000F465FF1F10B51721FFF7E0FF10BD000074
:1096E00070B50A000D00064B0221040000F08FFA4D
:1096F000060029782000FFF7D1FF300070BDC0467A
:10970000AB9A001170B586B000236A461370836867
:1097100004001D78681E0A2859D801A902F0C0F873
:10972000060633373B3F43474B4F5300180000F0CA
:1097300042F9062312284BD000281BD16088FFF77E
:10974000D9F90823002813D04279002A47D1264BA3
:109750001A78072312070BD5244B1A680723002A0F
:1097600006D01668002E03D0290001AAB0470300D6
:109770006A4613706B461B786088002B2AD1FFF76E
:1097800067FC06B070BD180000F06CF9D4E7180053
:1097900000F087F9D0E7180000F093F9CCE7180043
:1097A00000F0ADF9C8E7180000F0C3F9C4E71800ED
:1097B00000F0F6F9C0E7180000F0F6F9BCE7180071
:1097C00000F013FAB8E7180000F013FAB4E7072323
:1097D0006A46137069466088FFF782FFD1E7052368
:1097E000012AC5D1024BB8E78164FF1FEC65FF1F5A
:1097F000F065FF1FF8B52C4F8600F35904000D00EB
:10980000002B40D0DA8882423DD15A78062A33D1E3
:109810001A78002A2ED0012099681A6A097D01421F
:1098200006D0157B054203D007225A700120F8BDEF
:109830000220014204D0157B054201D00922F4E741
:109840000420014204D0127B024201D00B22ECE73B
:10985000164B1B68002BE9D05B68002BE6D020007C
:109860009847BB5900215B78122BDFD12000FFF70E
:1098700015FFDBE70E4BECE7112A04D1002900D0DD
:1098800032252900F2E7002D08D12000FFF732F938
:10989000002803D01023027913430371210028000C
:1098A000FDF798FAC2E7C046F465FF1FEC65FF1F9D
:1098B000F065FF1F70B50E4E8500AB590400002BFC
:1098C00013D01B78002B11D10A4B1B68002B04D03E
:1098D0005B68002B01D02000984773595B78122BEE
:1098E00003D100212000FFF7D9FE70BD024BECE749
:1098F000F465FF1FF065FF1FEC65FF1F094B80003B
:10990000C3581020002B0CD01A6A002A09D09B687B
:10991000002B06D0127A1B7E101C9A4200D9181C0C
:10992000C0B27047F465FF1F70B503000D0014004E
:109930000220002A30D000292ED013700B78081D89
:1099400053704B789370FFF7A7FCE0700120022161
:109950002B7A23716B7B034063716A7B0A4013434C
:10996000042263716E7B1640334363716E7BF6088D
:10997000F600334363712B7B0340A371287B0140C6
:1099800000200B43A371297B0A401343A3712A7B58
:10999000D208D2001343A37170BD10B50A000100B4
:1099A0000120FFF7C1FF10BD10B50A000100022021
:1099B000FFF7BAFF10BD70B506000C000220002EA4
:1099C00030D000292ED07378201D0B70B3784B70E7
:1099D000F178FFF76DFC01223579257271794B1012
:1099E000080013409340104003438810104080004B
:1099F000C9080343C9000B436373B1794B100800D6
:109A00001340934010400343881002409200C9085D
:109A10001343C9000B4321202373FCF773FE8542D7
:109A200001D2122070BD2220257AFCF76BFE854200
:109A3000F7D823781820042BF4D86378012BF1D8B9
:109A40000020EFE7030010B50220002909D0002B09
:109A500007D00322481C0A7019000D3201F088FE5D
:109A6000002010BD03000222080010B5002B06D014
:109A7000002904D00E32591C01F07AFE0022100099
:109A800010BD030010B50220002909D0002B07D01B
:109A90000422481C0A7019000C3201F069FE0020F3
:109AA00010BD10B5FFF7DEFF10BD03000220002936
:109AB00006D0002B04D0052200200A701B784B70C2
:109AC000704703000220002B08D0002906D05B78E5
:109AD00000200B70013B082B00D9183070470300A1
:109AE00010B50220002909D0002B07D00622481CFF
:109AF0000A7019000A3201F03BFE002010BD10B5BB
:109B0000FFF7B0FF10BD02000B00022010B50029C6
:109B10000ED0002A0CD007211970118859701188B5
:109B2000090A997011180822D81C01F021FE0020A2
:109B300010BD03000A00022010B5002B0CD0002934
:109B40000AD099785878090201431180901CD91CD9
:109B5000082201F00DFE002010BD030010B5022008
:109B6000002909D0002B07D00822481C0A701900D0
:109B7000921801F0FDFD002010BD02000B00022034
:109B800010B500290BD0002A09D0092119701178CD
:109B900018185970511C062201F0EAFD002010BD72
:109BA00010B5FFF75FFF10BD02000B00022010B5DB
:109BB000002A09D0002907D05178197011180622FF
:109BC000581C01F0D5FD002010BD030010B5022087
:109BD000002909D0002B07D00A22481C0A7019005E
:109BE000063201F0C5FD002010BD10B5FFF73AFFA9
:109BF00010BD02000B00022010B5002A06D000297B
:109C000004D018005178FFF753FB002010BDF0B5C9
:109C100085B017001E006A460623050008009181E2
:109C20009380FEF7C0FC1324011E02900CD0380074
:109C3000B047041E05D1280001A9FEF76FFA041EE3
:109C400002D0029801F0D4FF2800FFF701FA2000AB
:109C500005B0F0BDF0B504008BB0019115000021F6
:109C6000102202A801F004FF334EA700B8590028C3
:109C70003CD0C388A34239D10378002B36D1427837
:109C8000062A18D102000100553235310C3006ABDE
:109C9000FFF7A9FA002829D12000FFF72FFE0200C4
:109CA00006A902A801F064FD200002A902F060F8F4
:109CB00001200BB0F0BD816E002917D00B8A112A4C
:109CC00028D19D420ED101981231093A01F0D8FDF8
:109CD000012807D1BB5920009D6EFFF70FFE290018
:109CE0000200DEE732212000FFF7D8FC2000FEF75B
:109CF00001FF061E1BD0416A002918D00B8AAB4217
:109D000015D108220198123101F0BAFD01280ED1B7
:109D1000716A0AE09D42E9D108220198123101F0EE
:109D2000AFFD0128E2D1BB59996E8A7EB9E72000C8
:109D300001F0A6FEBCE7C046F465FF1FF0B56B4D11
:109D400087007E5985B0337802900393002B00D0B2
:109D500087E0B368346A01937078062817D101222E
:109D60001B7D134202D0217B114218D102221342E3
:109D700002D0217B114251D10422134203D0237B14
:109D8000134200D08BE0019B5A7DEB5991E00738DC
:109D90000428F8D801F084FD032E42678300B36ED7
:109DA000002B03D11C2001F033FFB066EB599C6EF1
:109DB000002C1CD010220021200001F059FE029836
:109DC000FFF79CFD01002000FFF72DFA01F078FD60
:109DD0002082200008211230FFF725FA0298FFF7B1
:109DE0008DFDA076EB592100D888FFF70FFC0822E3
:109DF000EB591CE0B36E002B05D01A00198AF088CD
:109E00001232FFF70DFC0222019B197DEB59114222
:109E10003DD0207B10423AD0073208E0F488FCF7AE
:109E2000DBFD01002000FFF711FC0A22EB595A70FC
:109E3000029B9C002A595378073B042B11D8D088E9
:109E4000FEF758FE00284ED0C3895A08D218284978
:109E5000029B0298CB542B5941180433254801F03A
:109E600037FF05B0F0BDFCF79FFD030001208342E2
:109E700001D100200393EB59DE88FCF79BFD039989
:109E800002003000FFF7ECFB019AEB59117D042230
:109E900011420CD0217B114209D00B22C7E7F68872
:109EA000FCF73CFD01003000FFF7EEFB6BE7019A89
:109EB000527D01210A4204D0607B084201D00C226D
:109EC000B5E702210A4204D0607B084201D00E228D
:109ED000ADE704210A4204D0627B0A4201D010227D
:109EE000A5E71222A3E7FA225200B0E7F465FF1FAC
:109EF000F865FF1FB3A2001110B5064B1A780423B2
:109F0000100018401A4200D00348FFF727FA00203B
:109F100010BDC0468164FF1F2C43FF1F70B50400B5
:109F2000FFF7D4FA051E43D12000FFF77FFA234E36
:109F3000A400A0598268937CDB0708D50321036A3B
:109F40001B790B40012B02D1017F0B430377431D8B
:109F5000D97F8B1E022B0DD8022900D00121C08889
:109F6000FCF790FF042133591A7F59700A431A777E
:109F7000280070BD01290CD102231022437000215A
:109F80000C3001F075FD305910213530FFF74BF9D9
:109F9000EEE70529ECD10223D118437010220C30D2
:109FA00001F0E6FB04233259117F0B431377EAE7F4
:109FB00008251828DCD1053DDAE7C046F465FF1F07
:109FC000F0B58BB0059143887E4F9E00F459150083
:109FD0000493002C15D1012902D000200BB0F0BD54
:109FE000101D57781678FFF757F9EB683200029387
:109FF0002B7A0499019300903B002000FCF70CFFA2
:10A00000EBE7E388049A934201D00820E6E723783F
:10A01000012B00D1D4E0059B581E092800D9CFE0C0
:10A0200001F03EFC05CE0A29CC506C859AB229007D
:10A030000498FFF773FFD1E7200029001022453074
:10A0400001F096FBB9594B78042B02D1013B4B70C0
:10A05000C3E70B000A00253335320C310498FFF7B3
:10A0600095F90498FFF702FA0522431E9841BB595F
:10A07000C0005A70B2E7200029001022553001F0CC
:10A0800077FB049B4F4C9D00295904980A0006ABAE
:10A0900055320C31FFF77AF929591022453106A8BB
:10A0A00001F0EEFB012808D10498FFF7F7F90590BD
:10A0B000002804D106222B595A7005988EE70823F0
:10A0C0000593FAE763780C2B7AD1E36E002B03D16A
:10A0D0001C2001F09DFDE066BB59D86E00286FD0B2
:10A0E0001022290001F044FBBB590498DC6EFFF7F5
:10A0F00005FC0D22A076BB595A706EE7E06E002871
:10A100005ED063780D2B5BD12B8808220382A91CBB
:10A11000123001F02DFBBB599A68517D0222114289
:10A1200026D0186A407B104222D00C32E4E76378D4
:10A130000E2B45D1236F002B03D1162001F068FDB3
:10A140002067BB59186F002803D01022290001F0A6
:10A150000FFB0F22BB59CFE763780F2B30D1206F55
:10A160000622691C103001F003FBBB599A68517D2F
:10A170000422114203D0196A497B1142D5D1002132
:10A180000498FFF78BFA28E7636F002B0DD0BB59BB
:10A19000586F0028F3D01022290001F0E9FA0122BB
:10A1A000BB5952425B6F1A61E9E7142001F030FDA0
:10A1B000BB5960675B6F002BE9D126E72978DFE7A1
:10A1C00007200BE7F465FF1F10B5064C207001F067
:10A1D000EFFA06212078FDF791FF0348FEF778FC9F
:10A1E00010BDC0460766FF1F6993001100200BB227
:10A1F00070B50D00834216DA264B187801F0E8FBA3
:10A20000041E0DD00378922B0ED0A02B37D0224BFA
:10A210001878FF283AD0210001F09AFD002835D1A6
:10A2200080200002684070BD43780E2B0BD03E2B7F
:10A23000EDD18378052B12D0082BE8D18179808865
:10A24000FFF7D8FA08E0154B82889A42DFD183687D
:10A250001878591CFEF7C0FE002817D1D7E7104B1D
:10A260001B785B0712D50F4B1B68002B0ED09B6829
:10A27000002B0BD0C289811D80889847ECE7FFF73F
:10A2800041FAA068002801D001F0B2FC200001F0E2
:10A2900067FCC5E70766FF1F2543FF1F1820000066
:10A2A0008164FF1FF065FF1F10B50078FFF712FAF9
:10A2B00010BD10B50078FFF7FDFA10BD0C23434325
:10A2C000084A10B59B185A68002A03D0012901D109
:10A2D000904710BD9B68002BFBD00029F9D198470F
:10A2E000F7E7C0462466FF1F01238340094A10B5E3
:10A2F000946B1C439463506B98435063D46B200061
:10A300009843012901D120001843D063116B0B43FE
:10A31000136310BD00800040F0B500240127154BE9
:10A3200085B0DA6B144E03921A6C0192DA64019BC9
:10A33000E3403B4217D0039DE5403D400295E5B226
:10A3400002992800FFF7BAFF316A736A002908D022
:10A350003900002B01D0029979402800FFF7C4FF93
:10A3600001E0002BF9D101340C36172CDFD105B0F8
:10A37000F0BDC046008000400866FF1F064B01216B
:10A380005A68C2400A4204D01B68C3401800084003
:10A3900070471B6DF9E7C046008000400122064B64
:10A3A0008240002903D0D9680A43DA607047D9682F
:10A3B0009143D960FAE7C0460038004030B5032425
:10A3C00044430F4BE25C1B199C785D7801232D1BE5
:10A3D0000135AB40013BA340A140DB430C001228F8
:10A3E00007D808499200521811681940214311609A
:10A3F00030BD054A11680B4023431360F8E7C0469F
:10A4000083C0001108F0004014F00040C21F70B576
:10A41000D4B20623092C0BD80125084C95400029FD
:10A4200008D00021FFF7CAFF23682B4323600023D5
:10A43000180070BD2368AB43F8E7C0460038004001
:10A44000214BF0B51B185B78022B21D10324444328
:10A450001E4A1F4EA35C12199478012215008540F4
:10A46000B76B013CE4B23D43A240B563194C1228DE
:10A4700015D89B0000290CD117495B1899680A432D
:10A480009A600123205C154A834011680B431360D6
:10A49000F0BD11495B18996891439960F1E70E4B43
:10A4A00000290DD159690A435A61225C1328E8D06A
:10A4B0000123203A93400A49086803430B60E7E709
:10A4C000596991435961F0E70866FF1F83C0001185
:10A4D00000800040C8C0001100F00040A0F0004023
:10A4E000A4F00040F8B500241B4E1C4D1C4B1B5D16
:10A4F000012B1FD1194A9269E2401A420BD0012266
:10A50000B25693402200143AD2B2022A09D8154911
:10A510004A6913434B61013402360C35172CE5D1DF
:10A52000F8BD0022B2560F499200521891680B43B1
:10A530009360F0E7022BEED1E7B23800FFF71EFF81
:10A5400001235840C1B23800FFF77AFF3800FFF707
:10A5500015FF6877DFE7C04655C000110866FF1F8A
:10A560000966FF1F00F00040012202388240054BBF
:10A57000002903D059690A435A61704759699143C8
:10A580005961FAE700380040F8B50E0001210F00CC
:10A590008740114A0400D368FD43BB43D360831E48
:10A5A0008B4201D8FFF7E0FF00212000FFF72EFFCC
:10A5B0000A4A0B4B5168012E05D139431B195160D2
:10A5C0005E700020F8BD2940516002221C196270A3
:10A5D0009A6915409D61F4E7003800400080004012
:10A5E0000866FF1F012210B58240074B002906D0E4
:10A5F00019680A431A600121FFF7C6FF10BD1968E8
:10A6000091431960F7E7C046008000400C2370B505
:10A61000002543430A4A29009B181D70094B04007A
:10A620001B185D70FFF7B0FF0123A3400649280007
:10A630000A681A430A6005490A689A430A6070BDAD
:10A640002466FF1F0866FF1F3480004030800040F2
:10A6500070B504000E00FF2813D003250540FFF756
:10A66000D5FF084AA3089B009B183F22ED00AA4093
:10A67000AE40196820009143314319600121FFF772
:10A680008DFE70BD18380040F8B50C244443134BC0
:10A690000500E4186368002B03D1A3681220002B87
:10A6A0001AD0022201270E4B00215B195A70280094
:10A6B0002770FFF769FF63681E1E08D0A3683E007D
:10A6C000002B04D02800FFF759FE4640F6B22800C0
:10A6D0003100FFF709FE0020F8BDC0462466FF1FC9
:10A6E0000866FF1FF7B5C420FF222B4B80001958C6
:10A6F000002491433F3A0A431A508022274F5202C6
:10A70000274E1A60274B1D5D002D21D0A31E012B63
:10A7100003D80121E0B2FFF727FF012D18D11F4B0D
:10A720009B69E3402B4213D0E3B218000193FFF77B
:10A7300025FE01000198FFF755FFE3B2143B022B01
:10A740001DD801217156184A8D405369AB4353619E
:10A750003B7F002B0DD0E5B22800FFF795FF2800C6
:10A76000FFF70CFE7B7F0100834202D02800FFF739
:10A77000A5FD01340C370236172CC3D1F7BD0121DA
:10A7800000237156F3568D40074A9B009B189A6828
:10A79000AA439A60DCE7C04600E100E00866FF1FBC
:10A7A00055C000110966FF1F00F0004070B50E0093
:10A7B00015000400FFF72AFF0C236343094A200019
:10A7C0009B189D605E60FFF75FFFF021064B074A14
:10A7D0008900051E5A5002D02000FFF717FF2800FD
:10A7E00070BDC0462466FF1F0000FF1F19A30011A3
:10A7F00070B5134D07202C78002C1FD19822210012
:10A800005200280001F02CFA0123C420FF222B70F3
:10A810000C4B80001C635C630B4B1C605C600B4B3F
:10A82000195891433F3A0A431A50802252021A6043
:10A830000D20074A074900F0F3FF200070BDC04615
:10A840000866FF1F00800040A0F0004000E100E02B
:10A85000E5A60011E5A40011030010B50620072BA2
:10A8600009D8054A137001F063F9D7210020034B82
:10A87000034A89005A5010BD5443FF1F0000FF1FB8
:10A88000951BFF1F70B51D0002240C2910D8094A22
:10A89000CA40D2070CD5FBF741FF041E08D1059A28
:10A8A00004992800FBF756FFFCF7C4FDFFF724FBD3
:10A8B000200070BD1210000030B50D7802232C006E
:10A8C0009C43184201D02B431C0008252300AB43B6
:10A8D000284201D02B00234320241D00A543204201
:10A8E00001D01C4325002A230D70184204D0117892
:10A8F0001E3B0B43137030BD0028FCD10C21137894
:10A900008B43F7E7F8B51D0006AB1B88140007AAB8
:10A910000E000B201778002B27D10A78022A49D184
:10A920004A68507811780002244A084380180428A5
:10A9300040D800F0B5FF03121D1B2300F06801F0A2
:10A94000BFF9021CC0B2B84200D93A1CD2B22000F2
:10A95000F1682A8000F00CFF06E00222F3681B88F1
:10A960002A8023701B0A63700020F8BD0622EEE7E0
:10A9700001232B80F3681B782370F5E7F368002B25
:10A9800016D008222A801A8822701A88120A627049
:10A990005A88A2705A88120AE2709A8822719A889C
:10A9A000120A6271DA88A271DB881B0AE371DBE7A5
:10A9B0002B80D9E701202B80D7E7C04600D6FFFFC8
:10A9C000F7B516000A781D0008AB1F880C0001239C
:10A9D000022A18D14A685078117800022B4A08439D
:10A9E000801803280FD800F05BFF02254439E06887
:10A9F00001F066F9C0B20723B84204D37B19019372
:10AA0000152B02DD0D231800FEBDE0682A00310081
:10AA1000C01900F0ADFE6B4600209B88E268D05460
:10AA20001B4B1B68834203D01B68834200D09847AE
:10AA30000023E8E70B23002FE5D1022DE2D1737844
:10AA400032781B021343E2681380114B1B68002B02
:10AA5000EED01B68002BEBD00120E8E70B23002F82
:10AA6000D1D1062DCED12A003100E06800F080FE61
:10AA7000DEE70B23002FC6D1012DC3D13278753309
:10AA8000012AC0D8E3681A70D2E7C04600D6FFFF9B
:10AA90001468FF1F70B50C001500072837D800F0A8
:10AAA000FFFE041436361B36242E182015290BD829
:10AAB000184E16220021300000F0DAFF2200290093
:10AAC000300000F055FE002070BD18200229FBD197
:10AAD0001288114B1A80F6E718200829F4D10A00D1
:10AAE0000E48290001F01CF9EDE718200129EBD1EF
:10AAF0000B4B10780B49DA69FFF7DEFEE3E718200D
:10AB00000129E1D1064B10780749DA6BF4E70220FE
:10AB1000DAE7C046FC67FF1FD243FF1FC843FF1F91
:10AB20005843FF1F8043FF1FA043FF1F030010B5C2
:10AB30000020DB0704D50721024A034800F08CF807
:10AB400010BDC046E0C000115843FF1F054A030076
:10AB50001068002803D082889A4201D1806870472B
:10AB60000068F6E70C6AFF1F0A88030008009A4293
:10AB700004D08A8804309A4200D000207047000038
:10AB8000F8B5F22200230D4F0D4E796805004243BF
:10AB90003370994200D07B600A4C0021200000F005
:10ABA00067FF00231A007C60AB4202D100203370A3
:10ABB000F8BD01332280DBB2F234F5E7046BFF1FEE
:10ABC000026BFF1F106AFF1F73B56B4601900600F2
:10ABD000684615001980FCF75FFF041E11D1002D97
:10ABE0000FD07689002E11D00C2001F011F800282A
:10ABF0000ED0084A0460136886808560002B02D15D
:10AC00001060200076BD1A001B68F7E70224F8E701
:10AC10001324F6E70C6AFF1F012100220A4B10B52E
:10AC200049420A4C198099809A719A70084B207099
:10AC3000012019805A60FFF7A3FF2078FCF78AFFF4
:10AC40000448FDF745FF10BD1C68FF1F0C6BFF1F7C
:10AC5000046BFF1F05AD0011022310B5002802D0C0
:10AC6000FFF7B2FF0300180010BD0000030010B58D
:10AC70000020DB0704D50421024A0348FFF7A4FFA4
:10AC800010BDC046F4C00011D843FF1FF0B50E261A
:10AC900087B003930CAB1F8802ABF61805000800C1
:10ACA00031000292FDF77AF804000120002C0FD049
:10ACB0003088FFF74BFF03000E20002B08D05E68A2
:10ACC000002E05D021002800039B029A0097B04770
:10ACD00007B0F0BD0A4B10B5984207D101220023FE
:10ACE00052420A808B708A808B7110BDFFF73CFF47
:10ACF0000028FAD001235B42038000238370F4E72D
:10AD0000FFFF0000F8B5050001290AD1134E002409
:10AD10003388F227AB4219D028001149FFF7DAFF38
:10AD200006E0022904D10139FDF750FF0028EDD0DB
:10AD3000F8BD3B0063437268D018D35A002B09D08A
:10AD40003A00002100F094FE0134E4B2054B1B7878
:10AD5000A342EED801235B423380DDE7046BFF1F83
:10AD60001C68FF1F026BFF1F10B5FFF7FDFE0300FD
:10AD70000020834200D0987810BD0000F0B589B063
:10AD80001C000EAB80CB03901E8810AB1B78049286
:10AD900002930B7A0D00DB0616D42B780593022B59
:10ADA00024D00498FFF7D2FE002812D003689C46F6
:10ADB000002B0ED0029B2200019329003B00644629
:10ADC00003980096A04705E00498FFF7BFFE00280F
:10ADD00002D10E2009B0F0BD8368002BF9D00A2201
:10ADE0002900039898470028D7D0F3E76B68587874
:10ADF0001A786B4B000210439842D2D8043B984219
:10AE000010D2684B984242D015D8674BC018012821
:10AE1000C7D80B20002EDDD1EB681A7859683A802C
:10AE2000200028E0614BC018032800D979E000F029
:10AE300037FD846A789E5E4B9842B2D10B20002E7B
:10AE4000C8D101233B80EB6831001B7823706889EF
:10AE5000013080B2FCF7A2FF3A88031E0ED00178C1
:10AE600002328A183A80428962704289120AA270BC
:10AE700059680278E01C00F07BFC06E004323A805E
:10AE800031000422601C00F0F3FD0020A2E70B203B
:10AE9000002E9FD1EB6807A91E8804233B80330A4C
:10AEA000300026706370FCF779FF051E28D004ABD4
:10AEB0009A890E2304A95B183E49C668FCF7E2FF95
:10AEC00000280BD12B783C486A680599FBF798FB62
:10AED000002803D1012304AA5B42D3813278022ADD
:10AEE00006D17168201D00F043FC3B8802333B8093
:10AEF0000E2304AA9B181B88A3701B0AE370C4E7E7
:10AF000004ABDE81F4E70B20002E00D062E7E96895
:10AF10000398FFF729FF02233B802070000A60702E
:10AF2000B3E70B20002E00D054E70222EB681B8809
:10AF30003A8023701B0A6370A7E7E86800F0C0FE40
:10AF4000C2B203000720B24200D243E70DD00299FB
:10AF5000DBB27118994202DB921BD3B20293029BBF
:10AF6000E9681A003B8089195AE70023F6E70B20AD
:10AF7000002E00D02EE70722EB683A801A78227064
:10AF80005A7862705A88A2705A88120AE2701A7946
:10AF90002271DA886271DB881B0AA37175E7C046EB
:10AFA000042900000228000000D8FFFFFFD6FFFFA1
:10AFB00003280000FFFF000024C00011F0B58DB091
:10AFC0006B460020089120229B5E83423DDAA64B0F
:10AFD000187800F0FDFC071E32D00378B02B2CD17E
:10AFE0000079023816281FD800F0D2FE17001E0084
:10AFF0001E001E0031001E0096001E001D011E00D6
:10B0000052011E0073011E00CD011E0050021E00E1
:10B010001E001E008E021E00E302944B94491B8802
:10B0200078880B80FBF72CF83800FCF7ADFF914BCC
:10B030001B68002B01D038009847380000F090FDC5
:10B040008020089B0002434018000DB0F0BDEE22A6
:10B050000021874800F00CFD0BAA3B7B79893889D9
:10B0600000923A000D32FCF7B1FD0400804B1B78D2
:10B07000002C3FD146E0804B788805937F4B410000
:10B08000CB5A0BAE073BDBB232880293002301930D
:10B090007B4B210006930093059BFFF76FFE744DD9
:10B0A000002810D1069B3A8A1B889A420BD138009F
:10B0B0000599123000F0E4FB002804D02B78628957
:10B0C0009B00EB185A80162306A81B183288200014
:10B0D0007989FCF7D7FE2B7804009A00AA185188CA
:10B0E0000029C3D00133DBB22B70002807D006A99A
:10B0F000C98A9180634A12889A42BCD802E0012131
:10B1000049429180002B04D059497888FAF7ECFF26
:10B110008AE73E890A2479E000253E89574B069349
:10B120007B88069A5B009B5A033B9D4202DB002D05
:10B13000F0D05BE0162206A812183B7B79890092BA
:10B140003A0030000D32FCF741FD0590002858D040
:10B150004689017A7888FCF703FD041E44D1464BEA
:10B1600078880793069B4100C95A454B0439C9B2F8
:10B1700006AAD28A06930291019400930599079B2F
:10B18000FFF7FCFD041E2FD1069B39491A88931C3A
:10B19000002D26D14B807988384B4900CB5A511964
:10B1A000033B8B4220DD059B31485B8941190B71C4
:10B1B000A91C0135C9B2EDB2059145191B0A2B71C5
:10B1C000059B2D490433181800F0D2FA2C4B059A30
:10B1D0001B88D318DDB22C4B9E4205D00136B6B287
:10B1E0009CE749889942D6D0002D0CD0204C2800ED
:10B1F000618800F0EDFC207021007888FAF784FF68
:10B2000012E7059CF0E7002C00D183E77B78142B34
:10B2100000D109E716493B794E800B700C71788894
:10B22000FAF724FF00E7162406ABE418210038895A
:10B23000FCF7B4FD011E00D1B7E1788822880F4CDD
:10B2400045002C5B0A4D013CE4B2029400240F4BF4
:10B2500001940095FFF792FD041E00D014E129002F
:10B260007888FAF761FFDFE60C6BFF1FC442FF1F0F
:10B270002468FF1F1868FF1F1869FF1F5464FF1F11
:10B28000086AFF1FC242FF1FFFFF00002668FF1F62
:10B29000162406ABE41821003889FCF77FFD011E57
:10B2A00000D182E178882288AE4C45002C5BAE4DFF
:10B2B000013CE4B202947C89AC4B01940095FFF709
:10B2C0005DFD041E00D0DFE029007888FAF736FF24
:10B2D000AAE60025A44B1D803B00F6331B78A24A4A
:10B2E00078880792AB4208D99E4B1288069306993C
:10B2F00043005B5A013B9A4203DB0799FAF728FFA8
:10B3000092E616246B00FB18059306ABE418059B28
:10B3100021001889FCF742FD011E03D1059B012481
:10B320001E8973E77888924B2288069C0993430014
:10B330001B5B904E013BDBB202930023009601930E
:10B34000099BFFF71BFD041E02D0059B1E895DE7CC
:10B350007B88069A5B009B5A079A108832881218DD
:10B36000934202DC1B1A013B33807F4C023032884F
:10B370000999001900F0FCF92388328801359B18DF
:10B380002380EDB2A8E70BAA3B7B7989388900922C
:10B390003A000D32FCF71AFC00250590059B002BA6
:10B3A00004D10A24002D00D16EE060E0059B78886E
:10B3B000197AFCF7D5FB0100041E63D1694C6C4B74
:10B3C000788806940993069B4400E45A694B063C2E
:10B3D000E4B20BAE32880793029401910093059971
:10B3E000099BFFF7CBFC041E4CD1079B5E491B88D1
:10B3F0001A1D002D30D14A80059B5B4C5A89631978
:10B400001A716B1C9BB2E318120A1A71162306A854
:10B4100032881B1879890598FCF734FDFF21AA1C96
:10B420002E1D03350B00059092B2B6B2ADB20028C6
:10B4300003D006ABDB8AD9B21B0AA21865191171B9
:10B440002B714C4D301D2A884949201800F090F985
:10B450002B88F618B5B2A1E74988914207D17A88BE
:10B4600006995200525AEB18053A9A42C4DC3E4CF7
:10B470002800618800F004FC207021007888FAF729
:10B4800071FED1E5002DF2D13E89BFE6162606AB4E
:10B49000F61831003889FCF781FC3D000400FA35CC
:10B4A00000282DD0037A9B060CD400227B89398991
:10B4B000788800923A000C32FFF7E8FB041E10D0A7
:10B4C0003E8915E03088FFF741FB00281AD08368D9
:10B4D000002B17D02100122278889847041EE4D050
:10B4E000EEE72B78002B02D17888FAF74BFE002686
:10B4F0002B78002B00D097E5002C00D194E585E651
:10B500000124DDE70E24DBE7162506ABED18290044
:10B510003889FCF743FC041E47D0037A9B0611D4FC
:10B52000154A7B881188994203D01448814207D17B
:10B530001380134BF2261D780023D9B2A94221D3E0
:10B540000924A1E72888FFF701FB00282FD0836892
:10B55000002B2CD02100122278889847041EDFD0BF
:10B5600092E7C0465464FF1F2468FF1F2668FF1F30
:10B570001869FF1F086AFF1F046BFF1FFFFF000011
:10B58000026BFF1F31005943546801336018615A40
:10B590000029D2D13C0008342100F22200F0E8F862
:10B5A00021007888FAF7F6FD3EE501246CE70E24C9
:10B5B0006AE71D4B1A887B889A4231D07888FAF75F
:10B5C000F3FD31E5F223059851684343CD18C95A7C
:10B5D00000291FD03B7A012B0BD16C88AB8878886F
:10B5E000AA1D0094FFF752FB041E02D000233B72F9
:10B5F0002E88F2220021280000F03AFA00232B8046
:10B60000059B0133DBB20593084B05991B78064A6D
:10B610008B42D7D801235B421380002CCED0F5E5B6
:10B62000002634000596EFE7046BFF1F026BFF1F37
:10B6300070B504000E001500FFF796FA031E08D13E
:10B6400031000548FFF790FA03001120002B02D0CB
:10B650001C8000209D7070BDFFFF0000F8B50B4FEF
:10B6600006003B780D001400FF2B0ED00A2000F0DE
:10B67000C7F9011E09D0B12303800023468003715E
:10B68000C5800481387800F063FBF8BD1944FF1FC2
:10B69000F7B50F0008A90600088809A90B24098836
:10B6A000002821D10234022B1ED1557813782D02A7
:10B6B0001D432B008B4301937334002B14D1FB6883
:10B6C000300019000093FFF74FFB019C85420BD01F
:10B6D0002A0030000099FFF7ABFF041E04D12A00B6
:10B6E00030007989FFF7BAFF2000FEBDF0B50E7873
:10B6F00085B003900AA805880120022E0DD14C6860
:10B700002778647824023C43054FBC4205D1039856
:10B71000DBB201960095FFF7BBFF05B0F0BDC04658
:10B7200002290000034B10B51B68002B00D098477E
:10B73000FEE7C046106BFF1F07B501A8FFF7F2FF39
:10B74000044A05480021121A00F08AFAF8F794F822
:10B75000FEE7C046146BFF1F1C44FF1F00000000E3
:10B7600001B40248844601BC604700BFB532FF1FE8
:10B7700001B40248844601BC604700BFE94C0100A7
:10B7800001B40248844601BC604700BFADAE000072
:10B7900001B40248844601BC604700BF0D19FF1F79
:10B7A00001B40248844601BC604700BF4536FF1F14
:10B7B00001B40248844601BC604700BFC9260000AE
:10B7C00001B40248844601BC604700BF55490100EE
:10B7D00001B40248844601BC604700BF253AFF1F00
:10B7E00001B40248844601BC604700BF7530FF1FAA
:10B7F00001B40248844601BC604700BFA54F010068
:10B8000001B40248844601BC604700BF2526000001
:10B8100001B40248844601BC604700BF851F000098
:10B8200001B40248844601BC604700BF1531FF1FC8
:10B8300001B40248844601BC604700BF8D30FF1F41
:10B8400001B40248844601BC604700BF1D4B0100A3
:10B8500001B40248844601BC604700BF3919FF1F8C
:10B8600001B40248844601BC604700BFC9A900007A
:10B8700001B40248844601BC604700BF8D1200003D
:10B8800001B40248844601BC604700BFCD4C0100B2
:10B8900001B40248844601BC604700BFE54800008F
:10B8A00001B40248844601BC604700BF253BFF1F2E
:10B8B00001B40248844601BC604700BF0D5201003C
:10B8C00001B40248844601BC604700BF2951010011
:10B8D00001B40248844601BC604700BF65710100A5
:10B8E00001B40248844601BC604700BF156B0100EB
:10B8F00001B40248844601BC604700BF0139FF1F04
:10B9000001B40248844601BC604700BFD91B000057
:10B9100001B40248844601BC604700BF5136FF1F96
:10B9200001B40248844601BC604700BF4537FF1F91
:10B9300001B40248844601BC604700BF6DBC0000F2
:10B9400001B40248844601BC604700BF4D1F00009F
:10B9500001B40248844601BC604700BFF30E0000FA
:10B9600001B40248844601BC604700BFED38FF1FA8
:10B9700001B40248844601BC604700BF3D18000086
:10B9800001B40248844601BC604700BFE1170000D3
:10B9900001B40248844601BC604700BFED4A010083
:10B9A00001B40248844601BC604700BF5147010012
:10B9B00001B40248844601BC604700BF055E000038
:10B9C00001B40248844601BC604700BFB939FF1F7B
:10B9D00001B40248844601BC604700BFF54E010037
:10B9E00001B40248844601BC604700BF75A900004D
:10B9F00001B40248844601BC604700BFF937FF1F0D
:10BA000001B40248844601BC604700BF1D4D0100DF
:10BA100001B40248844601BC604700BFC94A010026
:10BA200001B40248844601BC604700BF691F0000A2
:10BA300001B40248844601BC604700BF7939FF1F4A
:10BA400001B40248844601BC604700BF11470100B1
:10BA500001B40248844601BC604700BFCD3AFF1FD5
:10BA600001B40248844601BC604700BF9DA90000A4
:10BA700001B40248844601BC604700BF154D010077
:10BA800001B40248844601BC604700BF091B0000A6
:10BA900001B40248844601BC604700BFE9280000A9
:10BAA00001B40248844601BC604700BF113BFF1F40
:10BAB00001B40248844601BC604700BFC5210000B4
:10BAC00001B40248844601BC604700BF85520100B2
:10BAD00001B40248844601BC604700BFC56D010047
:10BAE00001B40248844601BC604700BF79180000D9
:10BAF00001B40248844601BC604700BF014C01000C
:10BB000001B40248844601BC604700BFF53AFF1FFC
:10BB100001B40248844601BC604700BF5D170000C5
:10BB200001B40248844601BC604700BFDD660100E5
:10BB300001B40248844601BC604700BF951BFF1F4B
:10BB400001B40248844601BC604700BFC51D000027
:10BB500001B40248844601BC604700BF0D34FF1F9A
:10BB600001B40248844601BC604700BF434D010058
:10BB700001B40248844601BC604700BFB54C0100D7
:10BB800001B40248844601BC604700BFB14E0000CA
:10BB900001B40248844601BC604700BF2124000074
:10BBA00001B40248844601BC604700BF291C000064
:10BBB00001B40248844601BC604700BF7536FF1FD0
:10BBC00001B40248844601BC604700BF8B520100AB
:10BBD00001B40248844601BC604700BF350E000036
:10BBE00001B40248844601BC604700BF45510100D2
:10BBF00001B40248844601BC604700BFD949010036
:10BC000001B40248844601BC604700BF017F0000C8
:10BC100001B40248844601BC604700BF3D4B0100AF
:10BC200001B40248844601BC604700BF595201007C
:10BC300001B40248844601BC604700BF056A0000A9
:10BC400001B40248844601BC604700BF350E0000C5
:10BC500001B40248844601BC604700BF4550000063
:10BC600001B40248844601BC604700BFB70E000023
:10BC700001B40248844601BC604700BFF94C010092
:10BC800001B40248844601BC604700BF090E0000B1
:10BC900001B40248844601BC604700BFDD32FF1F8B
:10BCA00001B40248844601BC604700BFB3520100A2
:10BCB00001B40248844601BC604700BF3939FF1F08
:10BCC00001B40248844601BC604700BFDD52010058
:10BCD00001B40248844601BC604700BFA946010088
:10BCE00001B40248844601BC604700BF090E000051
:10BCF00001B40248844601BC604700BF35550000CE
:10BD000001B40248844601BC604700BF0124000022
:10BD100001B40248844601BC604700BFA13AFF1F3E
:10BD200001B40248844601BC604700BF810E000098
:10BD300001B40248844601BC604700BF21460100AF
:10BD400001B40248844601BC604700BF352EFF1F86
:10BD500001B40248844601BC604700BF594F01004E
:10BD600001B40248844601BC604700BF5125000071
:10BD700001B40248844601BC604700BF311B00008B
:10BD800001B40248844601BC604700BF456B010016
:10BD900001B40248844601BC604700BF393BFF1F25
:10BDA00001B40248844601BC604700BFEDA5000015
:10BDB00001B40248844601BC604700BF5522000020
:10BDC0000003010302020303040205000602070048
:10BDD000080009020A030B030C000D000E030F03F9
:10BDE0001003110313001400150316032D3C00115A
:10BDF000613C0011000000000200000002BE0011C2
:10BE0000192A0F180A000000F1590000FD24000053
:10BE100041460100D9810011EDA1001141760011C8
:10BE2000DD7F001119540011BDAF001165500011E4
:10BE30003D3E00116D3F001100000000161600008D
:10BE4000020000004CBE0011F4FFF3FFD2FC000022
:10BE5000AD40001100000000000000005475796141
:10BE60000042322E30003030313800676974687516
:10BE7000622E636F6D2F70767678005448303544AB
:10BE8000000000000200000098BE0011292A282AA4
:10BE9000272A262A252A242A0A180000E20400005C
:10BEA0007102000078EC0000050000007440000002
:10BEB0001027000060F0000004000000066400008D
:10BEC000204E000000000000060000005C4400005E
:10BED000102700006CEE00000700000005000000C5
:10BEE0001F501D00023CB40000011800200000009B
:10BEF000A10200003031323334353637383941420F
:10BF000043444546000000001D58001171580011BF
:10BF1000000000000200000020BF00116F2A6E2AFE
:10BF20001A18EAD8BC80F0FC600000000000000095
:10BF300000005F066B2F363D7D077F3F777C596E93
:10BF40007971AF066D4FC6CBEB0EEFCFEEC3A9668E
:10BF5000E9E8FA60D6F46CBCBEE0FEFCEE3E9A76F0
:10BF60009E8E000001A00000000000006410B71DBC
:10BF7000C8206E3BAC30D9269041DC76F4516B6B17
:10BF80005861B24D3C7105502083B8ED44930FF0D9
:10BF9000E8A3D6D68CB361CBB0C2649BD4D2D3868F
:10BFA00078E20AA01CF2BDBDFB349B5F80000080DC
:10BFB000001000000000000043620011CD78001165
:10BFC00067620011D57C0011EB620011AB7C00119F
:10BFD00061630011817C0011B3630011497E00117F
:10BFE0001B640011497E00114D640011037E001195
:10BFF00061630011397C0011D9630011E17D0011EA
:10C000000000000000000000BF640011E17D00118D
:10C0100021650011E5780011052A042A012A002A69
:10C020000229032801280028011800180000000038
:10C030000000000000000000000000870101020174
:10C0400002010102010203030401030101010101D4
:10C050000303020103000D000E0010001100130085
:10C060001401070108010A010B011C011D02040251
:10C0700005020702080219021A021C021D0301032D
:10C08000020317000201000504000807000B0A0064
:10C090001716001D1C010201010504010E0D0111FE
:10C0A00010011413011716011A19020201020B0ADA
:10C0B000020E0D02111002141302171603050403D9
:10C0C0000807030B0A030E0D0001020307090A0B00
:10C0D0000E0F101112141718191A1B1F20212200FD
:10C0E00005A90011C1A90011000000000200000014
:10C0F0002AC0001100000000EDB600110000000091
:08C100000200000028C000113C
:020000041FFFDC
:1000000000000000A53D001108BE001104BE001153
:100010004C61FF1F00000000000000000000000015
:1000200000000000000000000000000000000000D0
:1000300000000000000000000000000000000000C0
:1000400000000000000000000000000000000000B0
:1000500000000000000000000000000000000000A0
:100060000000000000000000000000000000000090
:100070000000000000000000000000000000000080
:100080000000000000000000000000000000000070
:100090000000000000000000000000000000000060
:1000A0000000000000000000000000000000000050
:1000B0000000000000000000000000000000000040
:1000C0000000000000000000000000000000000030
:1000D0000000000000000000000000000000000020
:1000E0000000000000000000000000000000000010
:1000F0000000000000000000000000000000000000
:1001000000000000000000000000000000000000EF
:1001100000000000000000000000000000000000DF
:1001200000000000000000000000000000000000CF
:1001300000000000000000000000000000000000BF
:1001400000000000000000000000000000000000AF
:10015000000000000000000000000000000000009F
:10016000000000000000000000000000000000008F
:10017000000000000000000000000000000000007F
:10018000000000000000000000000000000000006F
:100190000133FF1F6131FF1FC16601000000000035
:1001A000000000000000000000000000000000004F
:1001B000000000000000000000000000000000003F
:1001C000000000000000000000000000000000002F
:1001D000000000000000000000000000000000001F
:1001E000000000000000000000000000000000000F
:1001F00000000000000000000000000000000000FF
:1002000000000000000000000000000000000000EE
:1002100000000000000000000000000000000000DE
:1002200000000000000000000000000000000000CE
:1002300000000000000000000000000000000000BE
:1002400000000000000000000000000000000000AE
:10025000000000000000000000000000000000009E
:10026000000000000000000000000000000000008E
:10027000000000000000000000000000000000007E
:10028000000000000000000000000000000000006E
:10029000000000000000000000000000000000005E
:1002A000000000000000000000000000000000004E
:1002B000000000000000000000000000000000003E
:1002C000000000000000000000000000000000002E
:1002D000000000000000000000000000000000001E
:1002E000000000000000000000000000000000000E
:1002F00000000000000000000000000000000000FE
:1003000000000000000000000000000000000000ED
:1003100000000000000000000000000000000000DD
:1003200000000000000000000000000000000000CD
:1003300000000000000000000000000000000000BD
:1003400000000000000000000000000000000000AD
:10035000000000000000000000000000000000009D
:10036000000000000000000000000000000000008D
:1003700039B700110000000000000000000000007C
:10038000000000000000000000000000000000006D
:10039000000000000000000000000000000000005D
:1003A000000000000000000000000000151BFF1FFF
:1003B000000000000000000000000000000000003D
:1003C000000000000000000000000000000000002D
:1003D000000000000000000000000000000000001D
:1003E000000000000000000000000000000000000D
:1003F00000000000000000000000000000000000FD
:08183800206FFF1F4118FF1F84
:10184000024981F3088802F0CBFB0000206FFF1FE4
:1018500070B500241E491F4A1F484C6308CA1B0567
:101860001B0DE4188242F9D11C4B80228B630021AE
:1018700009201B4B920519621A4B1B4DDA671B4B53
:10188000DA688243DA609A68194802409A60112047
:10189000296002F091F8112002F06EF86B6C154A85
:1018A000112013406B64144B144A63431B0C1384C4
:1018B0000122134B9A7201F009FC124B1B78002B8A
:1018C00004D1114B1021187802F092FB70BDC04674
:1018D000000005408807054000080540FF010000A2
:1018E00000F0004004E100E0003800403CF000401F
:1018F000FFDFFFFFFFFDFFFFAE0600001C61FF1FC3
:10190000D061FF1FFE63FF1FFC61FF1F10B502F0D7
:1019100037F9072804D0122808D0022808D010BDB3
:10192000044A0420136B01331363F8E70220F6E73F
:101930001420F4E7FC64FF1FF8B507000C00260034
:101940002500503630785135002804D10300287026
:1019500058342370F8BD2978CA00481E8141A31865
:101960003800A25C5B68C9B2FFF7D0FF00280DD138
:101970002B78DA00A218013350602B703378044AB8
:10198000013B3370136A01331362D8E70123DFE7A9
:10199000FC64FF1F5C234343074910B5C9180B00C3
:1019A00058331B78012B05D1FFF7C6FF034A936A12
:1019B0000133936210BDC0463065FF1FFC64FF1FFA
:1019C00010B502F0CDF8064A0121130010CB4942B0
:1019D000D967044B136002F0D3F9200010BDC04654
:1019E00000E100E01000100010B5040002F0B8F8AB
:1019F000024B1C6002F0C4F910BDC04600E100E0DB
:101A0000431E5A425341A022F0B5D2015B4213401B
:101A1000154D164A40019B182A18127E8BB0019171
:101A2000002A1BD01A000832D46F0022E6B206AF9B
:101A3000E4B294420EDC2818C369002B08D0019947
:101A400002AA117106AA049202AA167303A8984763
:101A50000BB0F0BD1978B9540132EAE71A7D1A7853
:101A600006AB01261A70E6E7BC67FF1F0040004086
:101A7000F0B5254B04004001C25C85B0002A2BD094
:101A80001A18117E002927D0917E002924D01179BF
:101A9000022921D11689D788D168F51BADB22A1C3D
:101AA000102D00D9102292B2BE4217D1181801236E
:101AB00003710023C269C38003819A4206D068463D
:101AC000032103730171029301A890470820002CA1
:101AD00000D0192001F0FAFA05B0F0BD013C6542D2
:101AE0006C41A0256442ED012C40084D1B1864197F
:101AF000074D0633013A92B2AA42EDD01888461C2F
:101B00001E80085C2070F5E7BC67FF1F00400040A6
:101B1000FFFF00000F220E4B10B5986810400238EE
:101B20000A280BD801F0FEFF0D0A0B0A0A110A0A57
:101B30000A0A060002210020FFF762FF10BD012102
:101B4000F9E70020FFF794FFF8E7DB6FF6E7C04600
:101B5000004000400F220E4B10B59868104002382C
:101B60000A280BD801F0DEFF0E0A0B0A0A120A0A35
:101B70000A0A060002210120FFF742FF10BD0121E1
:101B80000800F9E70120FFF773FFF7E7DB6FF5E7E0
:101B90000090004013B5334C2378072B3DD8324BCF
:101BA0001A78324B002A39D18022196852020A432E
:101BB0001A60252001F0C0FE20232D4A11680B4336
:101BC000802113606B460422C90508680733104260
:101BD00028D080210422C905C86810422ED0802157
:101BE0002020C905CA688243CA6014221A701A7874
:101BF000002A2FD18021C905C86820320243CA605B
:101C000014221A701A78002A28D11A4B1A7D2278C9
:101C10005A601D221A705932DA6013BD1A681649CB
:101C20000A40C5E7086802430A6014221A701A784D
:101C3000002ACED01A78013AD2B2F7E7C868024338
:101C4000CA6014221A7019784A1ED2B21A7000297A
:101C5000F9D1C4E71A78013AD2B2C7E71A78013A43
:101C6000D2B2CEE75443FF1F1C44FF1F3CF000409C
:101C70004C43FF1F00200040FFFFFEFF564B70B596
:101C80001B68012B03D1554A936D0133936501F015
:101C9000DFFF534B534A1860534B544C1A600123D7
:101CA000534A1360534A13602378002B06D0062250
:101CB0005149524802F0D4F800232370504A514B46
:101CC00010681B78C1B2002B0ED14F4CC0B22378E4
:101CD0005BB2002B4FDB237824785BB264B21B0429
:101CE00024021B191B1813600B1C50294ED95023BA
:101CF000464A47491078DBB2FF2202284BD10868D8
:101D0000444C454D267890432A78964254D92278FF
:101D100024782E78023B5D10A31B6B435201D31A2B
:101D200010335B111843086002F0DAF8031F012B2F
:101D300045D83A4B1B78002B06D0394B1B78002B2B
:101D400002D0002001F014FFA122364B92009978B6
:101D5000354B4A431B689B18832292009B181B78C3
:101D6000033B012B03D8AF20400002F0E9F8012229
:101D70002E4BDA8270BD237824785BB264B2FF33D5
:101D8000FF341B0424021B190138ABE7CAB2022A34
:101D9000AED20223ACE70868254C264D2678904346
:101DA0002A78964208D9227824782D78023B5B1055
:101DB000641B63435201B2E72378DBB2B2E7022827
:101DC000D5D11D4B1B78013B022B03D91B4B1B7834
:101DD000022BCCD16C20C8E79809FF1FFC0FFF1F16
:101DE0004864FF1FFF3F0000141003404C64FF1FB6
:101DF0000C10034000100340D50BFF1F7211FF1F92
:101E0000B40003408C09FF1F680AFF1F490AFF1F27
:101E100094000340460AFF1F470AFF1FF908FF1FEF
:101E20002209FF1F300DFF1F3409FF1FBC0BFF1FCE
:101E3000440AFF1F450AFF1F1C09FF1F2309FF1F3C
:101E400010B501F08DFF0022014B1A8010BDC04675
:101E50004664FF1F10B502F0D3F8A121054A89009E
:101E60009478054A61431268044B5218528C1A80C8
:101E700010BDC046300DFF1F3409FF1F4664FF1F11
:101E800010B50D4B0D4A9978A1239B004B43126866
:101E9000D218531DD97F0A4B1B88994209D2441C82
:101EA00007D0C82805D0D2695B1A5A43054B534363
:101EB000C01801F02DFF10BD300DFF1F3409FF1FAA
:101EC0004664FF1F7102000070B5244D2B68002B83
:101ED00028D002F09DF82B68D8402B680400002B16
:101EE00027D001F075FF2B68D8401D4B1D4A99780B
:101EF000A1239B004B431268D118D25C91239B0015
:101F0000002A20D0CA580132CA50174B17491B6803
:101F10000868834214D3D23B181A012A1AD0144BF2
:101F2000186070BD02F074F8124B196801F090FF50
:101F3000D3E701F04DFF0F4B196801F089FFD4E79B
:101F40000D495B18E8E7CA500C4B1B68DB68E418C6
:101F5000201AE4E7F530FF30E1E7C0461C08FF1F18
:101F6000300DFF1F3409FF1F9C09FF1F4864FF1F2E
:101F7000A009FF1F1808FF1F2DFF3F005064FF1F1F
:101F800070B504000D00282916D10300A433C288BF
:101F90001B889B1A0B4A9BB293420DD906006A36E6
:101FA00005223100653001F023FE002804D1310004
:101FB000200001F09DFF70BD2900200002F038F8DC
:101FC000F9E7C046FE7F0000F8B50500012001F0EA
:101FD0001FFE134CA36AA26A9342FBD1114E3360D9
:101FE00001F04EFF10490300086010484268944613
:101FF0000F4A17680022BC4501D24268BA1A0D4840
:1020000002603268AD18A422E562606A520302439E
:102010006262094A1278002A01D00F3B0B60F8BDBA
:1020200000F00040340AFF1FE408FF1F28100040A2
:10203000180AFF1F1C0AFF1F1C09FF1F70B5802410
:102040001025E405A3682B43A36001F0F1FDA3680C
:10205000AB43A36070BD0000F7B5160080221C00E2
:102060001023D2050191916805000B439360002273
:102070005A4BD7301A6001F0E3FE9D232A002F004F
:102080009B00EB58CA3201210092FC37002B01D093
:102090000021009A386801F0FBFD2900009BCB313C
:1020A0001A784F4BD3351A604B780A781B021343CA
:1020B0008A7812041A43CB781B061343494A1BBA89
:1020C00013604B790A791B0213438A7912041A436D
:1020D000CB7931001B061343434A1BBA13606B785C
:1020E0002A781B021343AA7812041A43EB781B06C2
:1020F00013433E4A1BBA1360019A330213433C4A0E
:1021000013603C4B22001B1B9C4603293DDCB3089B
:102110009A0013005142B21A032A46D1354AE018F8
:10212000511A82784078120400020243E05C0433C2
:1021300002430A600022FF2B4BDDF0222E4B1201DE
:102140001A600F222D4B1A602D4A1368002BFCD009
:102150000023224A27491360091B321D0B191B68F3
:10216000043A180A23706070180C1B0EA070E370FC
:102170000434002AF2DC802210213B68D2050133AE
:102180003B6093688B439360F7BD6346D57898189E
:1021900093782D061B042B43157804392B4355786F
:1021A00004322D022B430360AFE7022A0AD1114A01
:1021B000E05C511AE2185278120202430A600433BA
:1021C0009BB2B7E7012AB5D10A4A521AE15C116005
:1021D000F5E7084959180A600433ACE700000440E9
:1021E0003C00044038000440340004403000044007
:1021F0000C000440000104400400044010000440AE
:1022000014000440F7B5150080221C001023D205ED
:102210000091916807000B4393600023654AD73013
:10222000136001F00DFE9D233E009B00F9583B001A
:10223000CA363200FC33002900D07FE0586801F034
:1022400027FD390032785C4BCB311A604B780A7825
:102250001B0213438A78AC4612041A43CB78281D1C
:102260001B061343554A1BBA13604B790A791B02AC
:1022700013438A7912041A43CB791B061343504A3D
:102280001BBA13604B7A0A7A1B0213438A7A120430
:102290001A43CB7A21001B0613434A4A1BBA136028
:1022A000009A2B021343484A13602200474B1B1B22
:1022B0000093009BCE785B1801938B7836061B0445
:1022C00033430E78043833434E78043136023343B7
:1022D000019E33600328ECDC0321A808431C9B000B
:1022E0002940800003292BD13849E5185E18A978C8
:1022F0006D78E35C09042D02294319433160030022
:1023000008330021FF2B2DDD314B324919600F219D
:10231000314B1960012327490B60304B19680029A4
:10232000FCD006211B680B40042B20D0802200200B
:10233000D20593680A318B439360FEBD01217DE78E
:10234000022908D121495D18E1184978E35C0902A6
:1023500019432960D3E70129D3D11C495918E35CFB
:102360000B60CCE71948181801600433CAE7002352
:1023700010490B606346002B0CDC3B00FC335A68B1
:10238000102101325A608022D205936801208B43CC
:102390009360D2E7009B9B181B68190A1370517059
:1023A000190C1B0ED37004235B4291709C440432C1
:1023B000E0E7C046000004403C0004403800044010
:1023C00034000440300004400C000440000104408C
:1023D00004000440080F00001000044014000440F2
:1023E00070B5061E19D002225A4B9B799343012BDC
:1023F00013D1594B1A78FF2A0FD15A78FF2A0CD1E2
:102400009A78FF2A09D1DA78FF2A06D11A79FF2AA9
:1024100003D15B79FF2B00D199E0504B0C201A7847
:10242000012A08D000224E4D1A7029780B00093B72
:10243000042B01D8212070BD4B1F012BFAD9454C2C
:10244000A37B042B00D982E0A279032A00D97EE085
:102450009A1ED2B2012A02D860881F2877D9002E8E
:1024600056D0012E73D1A0880128E3D0002907D1CE
:10247000581E032803D801F055FB121715122E70B1
:102480002978481E032811D80025364B1D602823C3
:10249000237501F05DFDA84227D0A580CAE702217F
:1024A0002970EDE70421FBE70321F9E7073901294A
:1024B000C0D82D490968C96A8906BBD52B49087857
:1024C0000028B7D1012A01D9002BB3D102230B7008
:1024D0008021274D263389012878237501F080FC5F
:1024E00080212878890101F083FD0123A380214BFD
:1024F0001B78002B0AD0FA2280211F4B92001B88E8
:1025000009025A431A4B187801F08AFD002092E71D
:1025100001F026FB2B78A680073B012B03D9174837
:102520002E7001F02DFD114B114C1A78002A06D0A7
:1025300080210022207889011A7001F051FC01F0FD
:102540001FFC80212078090201F04AFCDEE71220FE
:1025500071E7C046A60BFF1F6B09FF1F1A09FF1F7B
:102560001C09FF1F4809FF1F5064FF1F2309FF1F9D
:102570001B09FF1F2109FF1F2C09FF1F001000402E
:1025800010B5002901D001F0A3FC10BDF7B5604BD8
:1025900001919978A1239B004B435E4A0600146881
:1025A0001022E418D6235B00E0583623FF33E35CA7
:1025B00000279343222B41D1574B0F3A1A600760F3
:1025C000012501F02DFC019B1880E8235B00E35CF2
:1025D000002B01D0B34258DD0023504FFB70AD33C8
:1025E000FF33E3581A68002A03D09B88DB439B071C
:1025F0001DD03823FF33E35C002B18D09B235B00F6
:10260000E35C002B13D1D133FF33E35CB3420EDA2A
:10261000A4235B00E15AE018090A023101F058FBDB
:1026200023000122FE33013E01351A87FA70E823A8
:102630005B00E35C002B2AD0A8B2FEBD03683D001E
:10264000002BBED081880430090A023101F040FB22
:10265000D6235B00E3581F60B2E72300B133BA0012
:10266000FF339858013781880430090A023101F09C
:102670002FFBE8235B00E35CBB42EEDCE822F61AAA
:10268000ED1800235200A354A6E70027F1E720002D
:1026900001F09EFC00281FD0002E1DDD7319882636
:1026A00047190193B600200001F0B2FB5A308000B8
:1026B00020184068013581880430090A023101F090
:1026C00007FB200001F054FBA3590133A351BD4285
:1026D00002D0019B9D42E6D1114BE35C002BABD0B5
:1026E00095239B00E35C002BA6D00E4BE15A0029FA
:1026F000A2D00D4AA35C994202D90133A3549BE7AF
:1027000000231A212000A35401F002FC94E7C046E4
:10271000300DFF1F3409FF1F00140340E010FF1F9E
:102720005A020000720200005E0200000D4970B5FE
:102730004A6E0D4CD2038B69D20BA24206D80B4DC8
:102740000224AA4204D901F023FC70BD0224644291
:10275000E21815007E2425402242F4D0A3432B43E7
:102760008B61F0E700F000400A200000FC1C000034
:10277000F8B51D4B1D4F1A78002A10D1BA7B002ADC
:1027800002D101321A7003E0032AFAD0022AF8D0EB
:1027900001F0DEFB00220120154B1A70F8BD154B2D
:1027A000154D1C68154B9E7801232B702878C0B2FC
:1027B00000F09EFBBB7B002B0BD101F0F1FAA123B3
:1027C0009B007343E41883239B00E41823782B7049
:1027D000E4E7032B02D101F073FBF0E70020022BAA
:1027E000DCD101F0BDFBEAE71C09FF1FA60BFF1FB0
:1027F0002309FF1F3409FF1F490AFF1F300DFF1F68
:10280000F0B587B00EAD2F780FAD2D780593AC469F
:10281000634614000E4D0CAA12782E7803930D9B7C
:10282000009201932200059B029701F041FA2E705D
:10283000012C01D0042C08D1802206498B889343B7
:10284000054A1278D20113438B8007B0F0BDC04611
:102850001C09FF1F6C11FF1F7809FF1F0B001B3B9A
:1028600070B504003020E02B0DD81300E025493B63
:10287000FF3B9BB2ED00AB4205D8034B2000198211
:102880005A8201F00DFB70BD8410FF1F10B501F0DE
:10289000DFF9054B00205B68052B04D9034A526819
:1028A000D20200D4980810BD00100040FCE100E006
:1028B00070B501F055F90D4B1B68FC33DC691D6ADE
:1028C000FFF7E4FF6419844204D2094B01241B681A
:1028D000002B07D004220024064B1A70064A936985
:1028E0000133936101F04CFA200070BD5064FF1F6A
:1028F0009809FF1F2309FF1FFC0FFF1F70B50C4D28
:102900002B68FC335C6A01F02BF9FFF7BFFF2B68E3
:102910000025FC339B6AE318834204D2054B1B68F5
:10292000AB4200D1051B01F02BFA280070BDC04658
:102930005064FF1F9809FF1FD722044B92009B5839
:1029400010B5002B00D0984710BDC0460000FF1FF7
:1029500010B501F0CFF8FFF7EFFF2749274BCA6DFD
:10296000274C1A4084235B001343CB65254B1B681F
:10297000186A01F04DF9244B244A1A60244B254A69
:102980001A60A022244B52001A60244B187801F0E0
:102990001FF92000224901F003F90023A36002334C
:1029A000A360204B2049236003232048A36001F04B
:1029B000F7F810221E4BFF201A60802252031A6083
:1029C000802292031A60802212041A6001F0D0F86B
:1029D000012001F085F9FA20400001F049F9582062
:1029E00001F0AEFA134801F0B3F8012001F018F934
:1029F000072001F095FA10BD00F0004000FEFEFF38
:102A0000141000405064FF1F000003400180063D89
:102A1000BC00034034080000A40003404A0AFF1F22
:102A200071020000C3090000FFFF3F0028100040B2
:102A300000E100E030750000674E336888331B68A2
:102A400083F3088801F0A4F9644A654913680020FB
:102A50000B401360634B644A1B68934200D1A6E0AD
:102A600001F016FA0221614A13688B431360FFF7E5
:102A70006FFF5F4B5F4C1878C0B201F0B1F80023D4
:102A8000A3600233A3605C4B0120236001F0C0F817
:102A90000323A36001F0B4F9040001F0D9F80500A4
:102AA00001F0AEF9554B186001F082F8544B1968EB
:102AB000621A531EA14200D213008022D203934215
:102AC00001D39B029B0A3268D16AC90700D471E026
:102AD0004C491C0C09689BB24C4359432402090A17
:102AE000641803264849FC3293680A6847489B1AD1
:102AF000474A0768126847499B18474A9A18334063
:102B00009208DB190A600360042B03D901323340B9
:102B10000A6003600E684149A619300001F098F977
:102B20003F4F3E493B68C3183B603000019301F0C2
:102B300067F83C4E3068081838493060884205D93B
:102B4000019B01333B6001F05BF8316001F0F0F86C
:102B5000354B1B78002B0DD001F07AF8334B621BFC
:102B6000196812188A4232D24919091B091A3048C9
:102B700001F016F82F4E337A002B0ED001F068F8D2
:102B8000621BF1681218914224D94919091B091ACC
:102B9000294801F005F800233372284B83F3088895
:102BA00001F08EF8002001F073F901F049F801F00E
:102BB0006FF95CE7DC0199000234641A5900641A69
:102BC00009214B438033CB40A408E41889E7FA215C
:102BD0008900CCE71A49DBE75064FF1F1CF0004076
:102BE000FFFFC1FF0C0AFF1FB64121031000004088
:102BF000490AFF1F14100040C3090000100AFF1FFC
:102C0000340AFF1F380AFF1F200AFF1F280AFF1F70
:102C10001C0AFF1F240AFF1FC409000071020000E4
:102C20006008FF1F2C0AFF1F1C09FF1FE408FF1F7D
:102C300000100040740BFF1F3C10004000000020FB
:102C4000DC050000A022054B92009B5810B5002B1C
:102C500001D0984710BD01F003F8FBE70000FF1F0B
:102C6000A122054B92009B5810B5002B01D098472C
:102C700010BD00F0F5FFFBE70000FF1FA222054B8F
:102C800092009B5810B5002B01D0984710BD00F062
:102C9000E7FFFBE70000FF1FA322054B92009B58B4
:102CA00010B5002B01D0984710BD00F0D9FFFBE70D
:102CB0000000FF1FA422054B92009B5810B5002B6B
:102CC00001D0984710BD00F0CBFFFBE70000FF1FCD
:102CD00070B500F0BDFF4F4B186001F049F90400DA
:102CE000C30702D401F0A4F870BD00224A4B1A6059
:102CF0004A4B18780138042829D800F013FF032024
:102D0000181C2400200001F01BF80128ECD0444CD2
:102D10002378042B6ED101F093F90028E4D001F060
:102D20003FF9582001F00CF902232370DCE7200062
:102D300001F03EF8E9E7200001F00AF8E5E720009D
:102D400001F03EF8E1E7200001F03AF9DDE701F09B
:102D5000C7F80500012808D1324B1B78053B012B31
:102D600003D82000FFF76EFFD1E72D4B1B78022B15
:102D700001D0052B20D1022D28D12B4B9B7BAB43BF
:102D80001CD12000FFF76CFF264B18780128BED11C
:102D90006405BCD4244925224B7B034205D1233A48
:102DA00013405A42534126331A000B7D9342AED949
:102DB000322000F0A5FFAAE7022D07D1194B1B789E
:102DC000052B11D12000FFF759FFDDE7012D0BD1B5
:102DD000012B03D12000FFF75FFF98E7062B03D1FB
:102DE0002000FFF767FF92E7200000F039FF022D77
:102DF0008DD1C9E7032B04D10C4B987C00F078FFF0
:102E000072E7072B00D06FE7094B987B01F0D0F8F1
:102E10006AE7C0469C09FF1F9809FF1F9009FF1F22
:102E20002309FF1F1C09FF1FA60BFF1FBC0BFF1F61
:102E3000D40BFF1FFA210A4B0A4A49001A640A4AB6
:102E40005A500A4A04395A50094A08319A64094AC0
:102E50005A50094A5C315A50084ADA667047C046EF
:102E60000000FF1F0128FF1FFD28FF1FB128FF1FC3
:102E7000E123FF1F7127FF1F811EFF1F551EFF1F2C
:102E8000F7B50B0CFF270122009300233C001E0026
:102E90001D009446019089B262469A401000084095
:102EA00018413618B6B2FF2F02D1012E00D19FB2C1
:102EB000009802401A41AD18ADB2FF2C02D1012D8D
:102EC00000D19CB20133102BE6D10320012E07D193
:102ED000012D04D1019B2401E4191C700138FEBDB1
:102EE000102EFCD10238102DF9D00230F7E7000087
:102EF0008023F7B59C46264B264F01932649274A47
:102F0000274D284C284B02281AD1604638600868A3
:102F1000264E3040802636033043086001990978F8
:102F2000002909D11660224A2A60224A2260E02242
:102F300019689143A03A1BE08021C9021160F2E7B1
:102F400066463E600F68194E3E408027FF023E43B2
:102F50000E600199097800290DD1176001280ED162
:102F6000154A2A60154A2260E02219689143C03A46
:102F70000A431A60F7BD802189021160EEE7E02163
:102F80000F4A02432A600F4A22601A688A43F0E718
:102F90004B0AFF1FE0000340D800034090000340AD
:102FA000000003405000034040000340FFFFE3FFE8
:102FB0000280063D804508220180063D8066082289
:102FC0000080069880550822F8B51E4B80261A68A6
:102FD000002014003440324232D11A681A4F324372
:102FE0001A6001223B68063093433B6000F010FEFC
:102FF0000122164D2B681E432E603B680A261343A0
:103000003B608027BF00124B1B683B4211D1013E41
:10301000F6B2FF2E09D17E220E4B1C682B68E40B02
:103020001440934323432B6005E0082000F0F0FD9B
:10303000E9E7002EEFD180222B68600893432B60D4
:10304000F8BDC046C4F000405CF0004018F00040FD
:1030500068F0004060F0004010B500F0C9FE0121AA
:103060005820034A00F024FFFFF7AEFF10BDC04612
:10307000600AFF1F10B578220021034800F058FFB6
:1030800000F09EFD002010BD4467FF1F70B50400D6
:1030900000F066FD00230C200B4A010059438D18F7
:1030A000515C00290DD0A14208D1012300246B708E
:1030B00000F0DEFE00F064FE200070BD01330A2B3C
:1030C000EBD11224F6E7C0464467FF1F70B5040039
:1030D00000F046FD002319001D000D4A107800285D
:1030E00006D0A0420CD1557001310C320A29F5D11D
:1030F000002B0AD100F064FD00F042FE002070BDFC
:103100005078461EB0411B18EEE700F0B1FEF3E721
:103110004467FF1FF7B504000C20002384460E4DC2
:10312000019267465F43E85D7E19A04212D00028F5
:103130000BD10A4B9C4662461B7808331370019BE7
:1031400070707C557160B360FEBD01330A2BE8D10D
:103150000320F9E70720F7E74467FF1F4067FF1FD9
:103160008020F8B5484BC0051B68C1248360474BDD
:10317000FF251A68012313434361454BA4001A68D5
:10318000444B40211A60444B1A68444B1A60444B2C
:103190001A59AA431A51C52292009E58AE43314390
:1031A000802699509F583F49F6010F403E439E505C
:1031B0009E5880273602360A3043985080201A598C
:1031C00000020A4002431A5104341A59364E3F0491
:1031D000324080263A431A511A5936061202120A10
:1031E00032431A5108341A5980260A4002431A51B0
:1031F000C32292009F58B446AF4337439F509F5815
:10320000294E0F4007439F509F5837408026360471
:10321000374380269F509F5836063F023F0A374368
:103220009F50C0221F59AF433A431A511A591202F4
:10323000120A1643C6221E5192009C58AC436546A2
:103240002C439C509C5800250C4020439850C7208C
:1032500080001A58154C1140C02212020A431A501D
:10326000134B1B78DB08AB4201DC0020F8BD237850
:10327000002B06D0A368002B00D0984701350C34F2
:10328000EEE71220F2E7C0465043FF1F4C43FF1FFA
:10329000B0F000403C67FF1FB4F000403867FF1FEC
:1032A00000E100E0FF00FFFFFFFF00FF4467FF1F9A
:1032B0004067FF1F030010B51F2809D80722002010
:1032C0001340072404490A78A24313430B7010BD2E
:1032D00000230620F5E7C0464067FF1F054B06495F
:1032E0001B780A6805485B0702401B0B134300204C
:1032F0000B6070474067FF1F1CF00040FFFFC1FFDD
:1033000070B50C25FFF7EAFF0A4B1C780A4BE4085E
:103310006543ED18002C01D1200070BD2B78002BE7
:1033200006D06B68002B00D09847013C0C3DF1E7BC
:103330001220F2E74067FF1F3867FF1F1FB500210B
:1033400002220B0001910091052000F099FC02235C
:103350000B490A681A42FCD120230393039B5A1E8F
:103360000392002BFAD1074A1368002BFCDA0B24D6
:103370006C442000012100F0C3FD207804B010BD92
:1033800090C8004000C8004013B504000A4B0193E8
:10339000019B002B01D1112016BDFFF7CFFF2300A9
:1033A0000340044205D0052000F032FC019B013BA4
:1033B000EDE71800F0E7C046FFFFFF0707B500F094
:1033C000CFFB80220821D205936A0191002B01D105
:1033D0000739916202210C4A11600199481E01903F
:1033E0000029FAD103311160053101910199481E7C
:1033F00001900029FAD11160002B02D18022D20560
:10340000936200F0BDFC07BD00C00040F0B52D4C3C
:1034100089B02378002B4FD1FEF7D2FA02232A4F2E
:1034200003903A681A42FCD120230693069B5A1E49
:103430000692002BFAD1254E3368002BFCDA0120CE
:10344000FFF7A2FF011E02D0112009B0F0BD03005A
:1034500003220190009005AD9F2000F011FC032194
:10346000280000F04DFD02233A681A42FCD12023C7
:103470000793079B5A1E0792002BFAD13368002B43
:10348000FCDA0120FFF780FF0028DDD10398FEF76A
:10349000ABFAAA786B7811041B020B4329780B4313
:1034A00063601300113B0A49052B07D801239340A1
:1034B000A3600B60012323700020C6E780231B0359
:1034C000F6E7C0463843FF1F90C8004000C80040E0
:1034D0009808FF1F1E4B30B55A6818781D4B85B0F1
:1034E000D31859424B4101210093002300F0D8FB2F
:1034F000194B1A4A02259A6300221A6510325A653E
:103500008022C4219D65164B1648D202DA678900D5
:103510004258154B80241A4080231B041343435008
:10352000642341200393E40500F006FA402000F0F4
:1035300003FA6562039D6B1E0393002DFAD10323EA
:103540006362FFF73BFFA562FFF760FF05B030BD88
:103550004443FF1F95FFFEF700C80040050001FF30
:1035600004E100E000E100E0FFFF00FFF0B585B0FE
:103570000700FEF725FA022305002D4C22681A42A7
:10358000FCD120230093009B5A1E0092002BFAD1FD
:10359000284E3368002BFCDA0120FFF7F5FE0028E7
:1035A00003D01124200005B0F0BD234B236002237B
:1035B00022681A42FCD120230193019B5A1E0192DA
:1035C000002BFAD13368002BFCDA0120FFF7DCFE78
:1035D0000028E6D1194B1F60022322681A42FCD151
:1035E00020230293029B5A1E0292002BFAD13368C9
:1035F000002BFCDA0120FFF7C7FE0028D1D1104BC9
:103600002360022322681A42FCD120230393039BE8
:103610005A1E0392002BFAD13368002BFCDA0120EA
:10362000FFF7B2FE041EBCD12800FEF7DDF9B9E7B2
:1036300090C8004000C8004001000006A8C8004033
:103640000180000110B50020FFF790FF10BD0000C1
:1036500010B5064B18705960FFF73CFF002113208E
:10366000034AFFF757FD002010BDC0464443FF1F2B
:10367000D534FF1FF0B5040085B003920291FEF728
:103680009FF9882263035B0B52051A438023DB05F5
:103690009D6A8023274F0092BA68002601901B0381
:1036A0009A420CD9F82326001B041E401C4206D067
:1036B0008022214B52025E6219680A431A60002D73
:1036C0000BD100F04DFA02221C4B1A608023DB055F
:1036D0005A62013A9A6200F053FB0023039A934224
:1036E00020D1002D0AD100F03BFA144B03221D60BB
:1036F0008023DB055A629D6200F042FB8023BA689A
:103700001B039A4208D9002E06D000220A4B0C490E
:103710005A621A680A401A600198FEF765F900209B
:1037200005B0F0BD009A0299D2181278CA5401333C
:10373000D4E7C0463843FF1F00C8004000C0004027
:10374000FFFFFEFFF0B587B0029103920400FEF781
:1037500037F9019000F004FA802302250122234E5C
:10376000DB0535605D629A6200F00AFB204F3B6822
:103770002B42FCD120230493049B5A1E0492002B5D
:10378000FAD11C4D2B68002BFCDA0120FFF7FCFD61
:10379000002802D0112007B0F0BD2000039A029942
:1037A00000F0F6F9022304003A681A42FCD1202303
:1037B0000593059B5A1E0592002BFAD12B68002B0E
:1037C000FCDA0120FFF7E0FD051EE3D100F0C8F9A7
:1037D00080230322DB0535605A629D6200F0D0FA37
:1037E0000198FEF701F9E0B2D5E7C04600C00040FD
:1037F00090C8004000C80040F0B5802489B00600A1
:10380000FEF7DEF8E405A36A02250393029000F0B8
:10381000A7F90123304F3D606562A36200F0B0FA62
:103820002E4C23682B42FCD120230593059B5A1E66
:103830000592002BFAD12A4D2B68002BFCDA0120CF
:10384000FFF7A2FD002803D01124200009B0F0BD2D
:10385000244B2360022322681A42FCD120230693C2
:10386000069B5A1E0692002BFAD12B68002BFCDA1D
:103870000120FFF789FD021EE6D11B4B03211E60CC
:10388000030001900090202000F0FAF90223226842
:103890001A42FCD120230793079B5A1E0792002B44
:1038A000FAD12B68002BFCDA0320FFF76DFD041E14
:1038B000CAD100F055F980230322DB053C605A622F
:1038C0009C6200F05DFA039B002B01D1FFF776FDAF
:1038D0000298FEF789F8B8E700C0004090C80040A1
:1038E00000C800400100000694C8004007B500026F
:1038F00001910422000A01A9FFF724FF0EBD000078
:1039000073B5050005240B4AA3005B429B18196898
:103910006B46DE1D3000FFF7B3FA022804D133787E
:103920002B55013CEFD276BD052CFCD00128FAD1F5
:103930000230F8E7140900111F2807D8012380225C
:103940008340D20591680B43936070473F2808D8A5
:103950000123802220388340D20551690B435361F3
:10396000F3E75F28F1D80123802240388340D20555
:10397000116A0B431362E8E71F2807D80122802150
:103980008240C9058B6893438B6070473F2808D8F5
:103990000122802120388240C9054B6993434B6145
:1039A000F3E75F28F1D80122802140388240C90521
:1039B0000B6A93430B62E8E71F2810D880230200AC
:1039C000DB05153A1968012A06D8202291431960AF
:1039D00019680A431A60704701228240F6E73F28BF
:1039E00011D880230200DB05353AD968032A06D8AE
:1039F00010229143D960D9680A43DA60EBE70122CB
:103A000020388240F5E75F28E5D842238022181A43
:103A1000413B8340D205516A99435162516A0B433D
:103A20005362D8E710B50400012813D1A022184929
:103A300092050B685B015B0913430B60154B164A3B
:103A400019681140154A0A431A60402219680A434E
:103A50001A6010BD0028FCD101000A2000F060F9B6
:103A600021000B2000F05CF9C0220A4B920019687B
:103A70000A4340211A601A688A431A60B022044936
:103A800012060B685B015B0913430B60E1E7C0465C
:103A900014F000401CF000407F00FEFF80FD01009C
:103AA00072B6074A1368013313600422054B1A608B
:103AB0000023054A13608022D2055360FEE7C0460A
:103AC0007808FF1FC0F00040C4F0004005490B68B3
:103AD000002B05D1044A0A6004490A60044A1360B5
:103AE0007047C046140AFF1F841E0000380AFF1FDB
:103AF000C4F000400023034A1360034A1360034AE2
:103B00001360704754F0004040F1004044F1004021
:103B100002B4714649084900095649008E4402BC66
:103B20007047C04602B4714649084900095C490023
:103B30008E4402BC7047C04603B471464908400039
:103B40004900095A49008E4403BC70470000000038
:103B500001B40248844601BC604700BF8D110100DA
:103B600001B40248844601BC604700BF75A900004B
:103B700001B40248844601BC604700BFED6B010000
:103B800001B40248844601BC604700BFE927000039
:103B900001B40248844601BC604700BF9573010030
:103BA00001B40248844601BC604700BF2D6C01008F
:103BB00001B40248844601BC604700BFC1660100F1
:103BC00001B40248844601BC604700BFADAE0000AE
:103BD00001B40248844601BC604700BFEDA5000067
:103BE00001B40248844601BC604700BF891401004B
:103BF00001B40248844601BC604700BFCD4C0100BF
:103C000001B40248844601BC604700BF090E0000B1
:103C100001B40248844601BC604700BF018900002E
:103C200001B40248844601BC604700BFE5120100B0
:103C300001B40248844601BC604700BFDD3F00007C
:103C400001B40248844601BC604700BF85520100B0
:103C500001B40248844601BC604700BFC95C010052
:103C600001B40248844601BC604700BFE917010067
:103C700001B40248844601BC604700BF85120100C0
:103C800001B40248844601BC604700BF496D010091
:103C900001B40248844601BC604700BF21440000D3
:103CA00001B40248844601BC604700BFC56D0100F5
:103CB00001B40248844601BC604700BF9D6A000011
:103CC00001B40248844601BC604700BF79970000F8
:103CD00001B40248844601BC604700BFC115010021
:103CE00001B40248844601BC604700BF691101006D
:103CF00001B40248844601BC604700BF4DF9000092
:103D000001B40248844601BC604700BF613701002E
:103D100001B40248844601BC604700BF89370100F6
:103D200001B40248844601BC604700BFBDA3001136
:103D300001B40248844601BC604700BFD54401007D
:103D400001B40248844601BC604700BF0134010051
:103D500001B40248844601BC604700BF053401003D
:103D600001B40248844601BC604700BF8D82000058
:103D700001B40248844601BC604700BF5976010087
:103D800001B40248844601BC604700BF9DA9000001
:103D900001B40248844601BC604700BFC9A90000C5
:103DA00001B40248844601BC604700BFE9F6000048
:103DB00001B40248844601BC604700BF09340100D9
:103DC00001B40248844601BC604700BFF5350100DC
:103DD00001B40248844601BC604700BF6D0B01007E
:103DE00001B40248844601BC604700BFB3520100E1
:103DF00001B40248844601BC604700BFED68010081
:103E000001B40248844601BC604700BF156B010045
:103E100001B40248844601BC604700BFD9B000002D
:103E200001B40248844601BC604700BFCD0C0100CC
:103E300001B40248844601BC604700BFDD0A0100AE
:103E400001B40248844601BC604700BF89440000B9
:103E500001B40248844601BC604700BF090E00005F
:103E600001B40248844601BC604700BFE94C010030
:103E700001B40248844601BC604700BF21A900008C
:103E800001B40248844601BC604700BFBD5C01002C
:103E900001B40248844601BC604700BF016C0100C8
:103EA00001B40248844601BC604700BF116E0000A7
:103EB00001B40248844601BC604700BF01670100AD
:103EC00001B40248844601BC604700BF75F8000099
:103ED00001B40248844601BC604700BFE9D4000039
:103EE00001B40248844601BC604700BFDD0C0100FC
:103EF00001B40248844601BC604700BF85C1000090
:103F000001B40248844601BC604700BF3D71010016
:103F100001B40248844601BC604700BF53B90000A9
:103F200001B40248844601BC604700BFF90D01009E
:103F300001B40248844601BC604700BFB70E0000D0
:103F400001B40248844601BC604700BF79120100F9
:103F500001B40248844601BC604700BFA9D80000F4
:103F600001B40248844601BC604700BF19FA000052
:103F700001B40248844601BC604700BFBD0B01008C
:103F800001B40248844601BC604700BFC1A50000DF
:103F900001B40248844601BC604700BFD1AE0000B6
:103FA00001B40248844601BC604700BF6DF60000C2
:103FB00001B40248844601BC604700BFC1F700005D
:103FC00001B40248844601BC604700BFF9350100D6
:103FD00001B40248844601BC604700BF71B00000D4
:103FE00001B40248844601BC604700BF41B70011DC
:103FF00001B40248844601BC604700BF0D52010075
:1040000001B40248844601BC604700BFF9ED0000DE
:1040100001B40248844601BC604700BFE90B0100BF
:1040200001B40248844601BC604700BF8B520100C6
:1040300001B40248844601BC604700BF51B800008B
:1040400001B40248844601BC604700BF01D70000AC
:104050000200000026C0001101000000F8BD0011A0
:104060000200000022C00011010000009040FF1F6C
:104070000200000000BE001101000000CC61FF1F23
:104080000200000020C00011030000004061FF1F7B
:10409000120000000200000026C000110100000014
:1040A00040BE00110200000022C00011010000000B
:1040B0003DBE0011020000004ABE001103000000D6
:1040C0007B61FF1F0200000020C000110300000000
:1040D0009061FF1F0200000022C0001101000000DB
:1040E0003CBE00110200000048BE001103000000A9
:1040F0005161FF1F0200000020C0001103000000FA
:104100007261FF1F0200000026C0001101000000C4
:1041100084BE00110200000022C000110100000056
:10412000D941FF1F0200000096BE001101000000EF
:104130007BBE00110200000022C00011010000003F
:10414000D841FF1F0200000094BE001101000000D2
:104150009861FF1F0200000022C000110100000052
:10416000D741FF1F0200000092BE001101000000B5
:104170006BBE00110200000022C00011010000000F
:10418000D641FF1F0200000090BE00110100000098
:1041900066BE00110200000022C0001101000000F4
:1041A000D541FF1F020000008EBE0011010000007B
:1041B00061BE00110200000022C0001101000000D9
:1041C000D441FF1F020000008CBE0011010000005E
:1041D0005CBE0011020202020202000000000000A8
:1041E000141300009D4C0011634C0011F4BE00112B
:1041F00090011D0018001800FFFF070102030405CD
:10420000060201060000000000000000000000009F
:10421000000000000000000000000000000000009E
:10422000030000000200000026C000110100000091
:1042300014BF00110200000022C0001101000000A4
:104240009442FF1F020000001EBF00110100000089
:10425000C661FF1F0200000020C000110300000023
:104260003064FF1F0200000022C0001101000000A6
:104270009442FF1F020000001CBF0011010000005B
:10428000C861FF1F0200000020C0001103000000F1
:104290002864FF1F12006C6C00000000000000008A
:1042A00000000000080700000001000000000111EC
:1042B000FFFF0000504859360000000000000000D9
:1042C0000B000500F0000000B400002800280028C2
:1042D0003075A000A000A000A00000080008E001C8
:1042E000F00010001000100010001000100050002E
:1042F0005000500010001000D00700000000000027
:104300000F0001000500307507001000010081FF5B
:1043100000000000FF000000A5750011AD73001142
:104320003D710011FFFF0100FF000000C19F00115F
:104330003D9D0011559C0011000000000000000090
:1043400000000800040000003B0001085902E001E1
:1043500088212800FF0000000200000026C0001194
:1043600001000000ECC000110200000022C000119A
:1043700001000000D543FF1F020000001EC0001115
:1043800001000000FC67FF1F0200000022C00011B6
:1043900001000000D443FF1F020000001CC00011F8
:1043A00001000000D243FF1F0200000022C00011E4
:1043B00001000000D043FF1F020000001AC00011DE
:1043C00001000000C843FF1F180018001D009001E5
:1043D00002000003020200000200000026C00011DB
:1043E0000100000000C100110200000022C0001105
:1043F000010000001844FF1F0200000018C0001157
:1044000000000000000000000200000020C00011B9
:0A441000030000001C68FF1F20FFDE
:040000051FFF184180
:00000001FF
